:100000000C9444230C946C230C946C230C94D52DE9
:100010000C946C230C94302D0C946C230C946C2356
:100020000C946C230C946C230C946C230C94612E14
:100030000C946C230C946C230C946C230C946C2304
:100040000C94682C0C946C230C94362C0C94102C6F
:100050000C946C230C94F12D0C946C230C946C2355
:100060000C94B22C0C946C236841774186419541E5
:10007000A541B441C341D241E141F14100420F42A7
:100080001E422E423D424C425C426B427A428A42C0
:100090009942A842B842C742D742E642F6420543D7
:1000A00015432443344343435343624372438143E0
:1000B0009143A143B043C043D043DF43EF43FF43E9
:1000C0000E441E442E443E444D445D446D447D44E4
:1000D0008D449C44AC44BC44CC44DC44EC44FC44DF
:1000E0000C451C452C453C454C455C456C457C45C8
:1000F0008C459C45AC45BC45CC45DC45ED45FD45B6
:100100000D461D462D463D464E465E466E467F4692
:100110008F469F46AF46C046D046E146F14601476E
:10012000124722473347434754476447744785473C
:100130009647A647B747C747D847E847F9470A4809
:100140001A482B483C484C485D486E487F488F48C9
:10015000A048B148C248D248E348F4480549164986
:100160002749384949495A496B497C498D499E4933
:10017000AF49C049D149E249F349044A154A264AE0
:10018000374A484A5A4A6B4A7C4A8D4A9E4AB04A84
:10019000C14AD24AE34AF54A064B174B294B3A4B20
:1001A0004C4B5D4B6E4B804B914BA34BB44BC64BB2
:1001B000D74BE94BFA4B0C4C1D4C2F4C414C524C3D
:1001C000644C764C874C994CAB4CBC4CCE4CE04CC0
:1001D000F24C034D154D274D394D4B4D5D4D6E4D38
:1001E000804D924DA44DB64DC84DDA4DEC4DFE4DAF
:1001F000104E224E344E464E584E6B4E7D4E8F4E14
:10020000A14EB34EC54ED84EEA4EFC4E0E4F214F76
:10021000334F454F574F6A4F7C4F8F4FA14FB34FCE
:10022000C64FD84FEB4FFD4F10502250355047501E
:100230005A506C507F509150A450B750C950DC5068
:10024000EF500151145127513A514C515F517251A5
:1002500085519851AB51BD51D051E351F6510952DE
:100260001C522F524252555268527B528E52A1520A
:10027000B452C852DB52EE520153145327533B532E
:100280004E536153745388539B53AE53C253D5534B
:10029000E853FC530F54235436544A545D5471545C
:1002A00084549854AB54BF54D254E654FA540D5568
:1002B0002155355548555C55705583559755AB5567
:1002C000BF55D355E655FA550E56225636564A5660
:1002D0005E56725686569A56AE56C256D656EA564E
:1002E000FE56125726573A574F57635777578B5733
:1002F0009F57B457C857DC57F157055819582E580F
:10030000425856586B587F589458A858BD58D158E1
:10031000E658FA580F59235938594D5961597659A9
:100320008B599F59B459C959DE59F259075A1C5A69
:10033000315A465A5A5A6F5A845A995AAE5AC35A1F
:10034000D85AED5A025B175B2C5B415B565B6B5BCB
:10035000815B965BAB5BC05BD55BEB5B005C155C6C
:100360002A5C405C555C6A5C805C955CAA5CC05C05
:10037000D55CEB5C005D165D2B5D415D565D6C5D93
:10038000815D975DAD5DC25DD85DEE5D035E195E1A
:100390002F5E455E5B5E705E865E9C5EB25EC85E92
:1003A000DE5EF45E0A5F205F365F4C5F625F785FFF
:1003B0008E5FA45FBA5FD05FE65FFC5F126029606A
:1003C0003F6055606B6082609860AE60C560DB60C6
:1003D000F16008611E6135614B61626178618F6116
:1003E000A561BC61D261E961006216622D6244625E
:1003F0005A62716288629F62B662CC62E362FA629C
:10040000116328633F6356636D6384639B63B263C8
:10041000C963E063F7630E6425643C6453646B64F2
:1004200082649964B064C864DF64F6640D65256510
:100430003C6554656B6582659A65B165C965E06523
:10044000F865106627663F6656666E6686669D6628
:10045000B566CD66E566FC6614672C6744675C6725
:1004600074678C67A467BC67D467EC6704681C6812
:1004700034684C6864687C689468AC68C468DD68FB
:10048000F5680D6925693E6956696E6987699F69D6
:10049000B869D069E969016A1A6A326A4B6A636AA3
:1004A0007C6A946AAD6AC66ADE6AF76A106B296B69
:1004B000416B5A6B736B8C6BA56BBD6BD66BEF6B23
:1004C000086C216C3A6C536C6C6C856C9E6CB86CCF
:1004D000D16CEA6C036D1C6D356D4F6D686D816D6F
:1004E0009B6DB46DCD6DE76D006E196E336E4C6E05
:1004F000666E7F6E996EB26ECC6EE66EFF6E196F91
:10050000336F4C6F666F806F9A6FB36FCD6FE76F0D
:1005100001701B7035704F70697083709D70B7707B
:10052000D170EB7005711F71397153716E718871E3
:10053000A271BC71D771F1710B72267240725A723E
:1005400075728F72AA72C472DF72F97214732E738D
:10055000497364737E739973B473CF73E9730474CE
:100560001F743A74557470748A74A574C074DB7403
:10057000F67411752C75487563757E759975B4752B
:10058000CF75EB75067621763C76587673768E7647
:10059000AA76C576E176FC76187733774F776A7757
:1005A0008677A277BD77D977F57710782C78487859
:1005B000647880789B78B778D378EF780B7927794F
:1005C00043795F797B799779B379CF79EC79087A38
:1005D000247A407A5D7A797A957AB17ACE7AEA7A13
:1005E000077B237B407B5C7B797B957BB27BCE7BDF
:1005F000EB7B077C247C417C5E7C7A7C977CB47CA2
:10060000D17CEE7C0A7D277D447D617D7E7D9B7D56
:10061000B87DD57DF27D107E2D7E4A7E677E847EFC
:10062000A17EBF7EDC7EF97E177F347F527F6F7F95
:100630008C7FAA7FC77FE57F028020803E805B8021
:1006400079809780B480D280F0800E812C8149819E
:1006500067818581A381C181DF81FD811B82398210
:10066000578276829482B282010002000400080060
:100670001000200040008000000100020004000083
:10068000000000000000010201010303030303074F
:100690000B0406FE0805E905FF3C6EEBD11A1A08AB
:1006A000FD1413F00600ECFFF6DFF9FCC8D9F2CC1C
:1006B000C1D3D3BBC2D0B8B8C3C4C2BABFC5BFC30D
:1006C000CCCCC4CED5D7DBDEE8F2F7EFED052E2C8F
:1006D00006111C2755593A3E47454F5D656B6E6FB5
:1006E00071706F706D6A695A4846463F3C3A3731BF
:1006F0002B2926201B18140F0C0500FBF9F5EBE73E
:10070000E7E0DBD3CCD3C6BCC5BDB4AFADADA6A0CE
:100710009B9C9E9C9B9A9898969596969596979852
:10072000999A9D9F9FA5ADAFB0B2B6B8BEC4C6C9D9
:10073000CED1D6DBE0E5EAEDF1F5F9FE0205090DD3
:100740001217181E2627272E3A3B343E4E4D3F4F98
:100750007065556A756A686C6D6D6E6C6A6C6B68F5
:100760006562605B524F4E453C3B3A3734302B2B31
:1007700029211D1C18130E0B0803FEFAF8F3EEEBEB
:10078000E9E6E1DEDBD7D5D2CDCCCBC7C3C1C0BB58
:10079000B9B9B7B3AEAFB0ABA6AAADA8A2A1A3A397
:1007A000A1A1A3A4A4A2A4A4A0A5A7A4AAABA9A9FB
:1007B000AAAFB0AFB1B6B6B5B6BABEC1C5C5C6C9A7
:1007C000CACDD0D3D6D8DBDCDEE1E3E9EBEBEDF04C
:1007D000F2F2F7F9F8FE01FCFB030909070C110F0F
:1007E0000E12131214171A1A18181B1D1D1C1E2185
:1007F000201E1E1F1F212121211E1E2222222222F5
:10080000212122232323232325272527292828299B
:100810002C2B292C2E2C2B2E30302F30312E2E33FA
:1008200032302F2F2E2E2D2D2C2C2C292626242213
:10083000211F1D1C1B181614110E0C0B070504019B
:10084000FDFAF9F7F4F2F0EDEBE8E6E4E1DFDDDAEA
:10085000D8D6D3D1D0CECAC8C7C5C2C1BFBCBAB81A
:10086000B7B7B4B2B2B0AEACA9A9ABAAA9ACABA8A9
:10087000A8A9A8A8AAACACADAEAFB0B0B1B3B6B79A
:10088000B9B9BABFC1C4C8CACCCFD2D4D7DADEE3B3
:10089000E6E7EBF0F3F5F8FCFF0205090B0E111487
:1008A00016191B1E20232527292B2D2F31333434D5
:1008B0003537383A3B3B3C3C3C3D3E3C3B3D3E3D86
:1008C0003C3B3A3A3C3A36373836343332302E2EC7
:1008D0002C292828262423201E1D1C191715141224
:1008E000100F0D0B09080604030100FEFDFBFAF8CA
:1008F000F7F6F4F3F2F0EFEEEEEDECEBEAE9E8E810
:10090000E8E7E7E6E6E6E5E5E6E6E6E5E5E6E7E785
:10091000E7E7E7E8E8E8E9EAEAEAEBECECEDEEEF36
:10092000EFEFF0F1F2F2F3F3F4F5F6F6F7F8F8F989
:10093000FAFBFBFCFCFDFDFEFEFF000000010202D5
:10094000020303040404040505050605050606065E
:100950000606060606050505050505050404040446
:100960000403030303020202020101010101010168
:1009700000000000FFFFFFFFFFFFFFFFFFFFFFFF83
:10098000FEFEFEFEFEFEFEFEFEFFFFFFFFFFFFFF80
:10099000FFFF00000000000001010101020202034C
:1009A00003030304040404050505050506060606FD
:1009B00006070707070708080808080808080808BE
:1009C00008080808080808080707070707070707AF
:1009D00007060606060606060605050505050505BD
:1009E00005050505050505050404040404040404BF
:1009F00004040404040404040404040404030303BA
:100A000003030303030303030202020202020202BE
:100A100002020201010101010101010101010000C5
:100A2000000000000000000000000000000000FFC7
:100A3000FFFFFFFFFFFFFFFFFFFFFFFFFFFFFFFFC6
:100A4000FFFFFFFFFFFFFFFFFFFFFFFF00000000B2
:100A5000000000000000000001010101010101028D
:100A6000020202020202020203030303030303035E
:100A70000304040404040404040404040404040536
:100A80000505050505050000192926282826221F29
:100A900018060E03D2B4ACB19F9CA19EAAAFBBC7EF
:100AA000CDD0D3DDE4F10002142425413835585B64
:100AB0004F4235415844485A4A425B68596B5C374B
:100AC0005868452823201819130802F7F1E9DBD8E4
:100AD000D0C6C0B4AFA39592908B8894A69A8D90FF
:100AE0008F949691949C9EA9B5B7BDC5CBD0D6E204
:100AF000EEF3FD0708131F233B47536666757772B5
:100B0000716F6E6B6D68666053473F372D22140F0F
:100B100007FDF5EDE6E1D9CBCCC6BCB3AC9E95A5FF
:100B20009D8D91948D8B939490939FADACB8D1CFC4
:100B3000DEF3F4EAFD15142B1E1C2B1F3947465417
:100B4000535971665F6B5B625B5C6A5141372D275D
:100B50001D130C04FAE9E3E8DBCFCEC5C1B9B7B386
:100B60009DA7A6A2A6959BA29A9AA8A59CAAB3B255
:100B7000B0B0CADAC8C9DCECF7FAFE0A0906251AD1
:100B80001234333A2A253F4022152B262C282430B4
:100B90003D371C152B3C1B161E0E0E0FFEFAFEE6F3
:100BA000E7F4E0D8DCC9CFC9A9C6CBA6A9ADB2A8E5
:100BB00095BBB5A0C6C5B4CAD1D0DCE0EBECECED7A
:100BC000E9F5FDF6FA02050A11272A1E192A3E291F
:100BD00033443F474349534C484A472F2D3F281C35
:100BE00016151300FDF6F4F0E6DFDDD1CAD7BEC05E
:100BF000C4ACB4BAB7A6A3AEB7C1B7B1BFC5CED661
:100C0000C9D8ECDDE50205F60A201214161B2920CE
:100C1000251F192E271E2E30262222182C27162B90
:100C2000170D1818130C0B0B09F6F908F5F2ECE088
:100C3000F5EBDBE3E3E1E3DFCFE0D8D2E8DAE0DDB8
:100C4000DCE9DBE7E9E0EBEFE9F0F5EFFCFB0104C1
:100C5000F5FC13080314050A0B0908071004020D1C
:100C600006010F110C16151E241819192327252902
:100C70002218231E0D160E040AFDF8FEF4EFECE90F
:100C8000E8DAE0E1C9CFDAD4CBC5D4D5CAD3D6D41B
:100C9000D8E8E6DAF1F7E5FC00F40601060CFF0DF2
:100CA000170F0C13211F1B26181E3E29262E27293D
:100CB000202A2F231E171C1A0F11090305FFFA0102
:100CC000F6EDF4F1EDE8E3DDE2DED0D8D7D2D5D40D
:100CD000DBD1D3E3E5E1E2EAEAF1F9F1FC08FB0458
:100CE0000B0512130C13181815191B131A15131DC5
:100CF0001517161113111B0F03130E0A0D030A0FFC
:100D0000050503FD0408FEF5FBFEF8F9F6F2F5F41F
:100D1000F2EDF0F2ECF2F2EBF3F0EAF3F6F3F5ECCD
:100D2000EDFFF6F706F5F607FBFA02010500FE02F5
:100D3000030904010B06070F07060B0A060C0C0B30
:100D400014101212131810171811141514100C1077
:100D5000100D0B0503010200F9FCF7F2EFEEF1EEC6
:100D6000EAEAE8E8E8E8E6E4E7E9E7EBEDE8EEF4EC
:100D7000F4FBF7F80302030C09060B110E11130C18
:100D80000F14151919151715171D18120D161A0C11
:100D90001012090A0706050100FBF8F9FCF9F7F83B
:100DA000F3F5F5F4F6F2EEF0F4EEF0F0EBF0F1EF2F
:100DB000F0F8FAF8FBFEFE00080B0807070B110C11
:100DC0000A0D090C0E0E0D0D0F0B090506100A0475
:100DD00007040405050504030204070401020602D2
:100DE0000409030505FF06050102020300FD0101D8
:100DF0000000FEFDFD00FEFCFEFDFEFDFBFDFBF820
:100E0000F8FAFAFFFCF9FBF70003FE02FFFE01020D
:100E1000030202040808030C0C040B0C0B0D0E0C4F
:100E20000C0E0A0E0D0B0F0C0B0C0C0A0A0806090F
:100E3000040200FD01FEFDFCF3F8FAF5F7F3F2F50C
:100E4000F3F2F3F4F3F3F3F7FAF7F800FFFA02071B
:100E500000010A0A09070A0B0B0B0B100B0C1109F6
:100E60000A0B0A0C0909090707080506050104030E
:100E7000FF0001FFFDFEFAF9FDFBFCF9F8FCF8F6B6
:100E8000FDFFF9FBFBFBFFFFFF000200030503066C
:100E90000704050A090809090908090908070505D9
:100EA00007080403040203010101000202FD01011D
:100EB000FD01FDFC02000001000000010403030429
:100EC00003050505050509070408070406050706C7
:100ED00004050504010304FF000201FEFE0200FDFB
:100EE000FE0000FDFCFEFCFE00FDFCFFFDFF01FD21
:100EF0000003010204050705050809080B0C070992
:100F00000B08080A09080605060705050302020082
:100F10000100FD00FEFCFDFDFCFAFBFBFAFCFCFA07
:100F2000FAFAFDFDFBFDFDFDFEFF010201030403D6
:100F30000507050506060808070808070808050646
:100F4000050504020403FF000100FFFEFDFFFDFC98
:100F5000FDFDFDFEFDFCFDFEFFFEFEFEFEFFFE00B4
:100F60000201020202030504040504050605050545
:100F7000060504050504040303040302030200023A
:100F800001000000FFFEFFFE00FEFDFFFFFE00006F
:100F9000FF0000010102030403040504060705061F
:100FA00006070707070606060506070404040304E8
:100FB00003020101020000000000FEFEFFFFFEFF31
:100FC00000FEFE0000FFFF00000000010101020220
:100FD00003030304040405050505050604040504CC
:100FE00004040303020202010100010100FFFFFFEC
:100FF000FFFEFEFEFDFDFEFEFEFEFEFFFFFF00000B
:1010000000010203030304040404050505050504A7
:1010100005050404040403030302010101010000A7
:1010200000000DFE1B240400FFDDBBA6A6BEEA3BAC
:10103000777A622DFBCBADB3D8EFCCC3FC4B7348B2
:1010400005EDEAD2C7EA0F00DFE7F1F30B0AEBE1A7
:10105000FB151103F7EDEEF0F2EDD7E2FCE9CAB6AD
:10106000BCD7EB1C64723E04E4D9DAE1D2CAE1D603
:10107000B6C60A5B610FC9D10E2910F4E3DDEB118E
:101080002002061F03D0D4F8ECEEE3ABAFD1F73764
:1010900032E9E41E3520FDE5BDB2EBD9B6E00D4BDB
:1010A000560EE0E6EED3AFDC2B17EACCA8D30FDB6D
:1010B00095A0D82B74692EF5CBF212DCF43902BC62
:1010C000D2CDBCCEE938591EE7E408DF8F9BACA631
:1010D000D322677E6B2FE3A094CEE2CBBEB6F45C46
:1010E0007A7038EBD1A490E22A2D02BFAAD0F6295B
:1010F000552F1720E5A49FBEE30A2A25DA92B9E608
:10110000C6CDFADFBBF13F424024CFDDE19599D84F
:10111000114E6B3D1C455D16CADAEABF8FA7F42558
:10112000371BDCCED6B49BBCF7140B1F39FFBFAB0B
:10113000C50F261B373E17FBE4CCD6FAFFD9C5BC3A
:10114000C3F20A0A1D22F5C6CFD1BEEE2D382311F7
:101150000AF9D1AEBAF9454B0ACCCC1433DF9296DA
:10116000AED82F694401DADAFA191CEDBFC4E8FCE5
:10117000EE024E7A5709D9E6D4A0B2E0FB0502EDA3
:10118000CCD90D3330FFE2FC1E494E0DFD06D4C70D
:10119000F70F04D5A29FC5014F683F13CE9BBAF449
:1011A000FED4D3FEFD0B3116FA1D1CF5FEFDD4D581
:1011B000F1061804D2C6DED7BFD9204D3A15FAD4AD
:1011C000B6C3F1273B36412AEBBCAFD40F363719F3
:1011D000E5B1C7FFF9FE2B2DFBD3E304EFEA1C1E9C
:1011E000F9F0E3E0081D1B302CEBBEC3D608312A12
:1011F0000CCEC201171A3726E1B2CF17340CEB0020
:10120000EBBCDF0E02062C1FE9EB122624181D187A
:101210000601DEB1ACB9F23F4509E4001C1F1F080E
:10122000FBFFECDCEF0AFFDCCDDCF1FB090DF0FC91
:101230004E5F1DE2B7BCF1181B21302601E9E2DA4E
:10124000E6000D0F120EF7EA0C2407DFDBF8FCECCA
:10125000EDFC213919F6FDFDF7F5F40806F4F1ED82
:10126000FD0800FBFAFC05110FFEFBFDF6F40F2D47
:101270001AEACED7FA06F7F5FDFA01161A0EFBEEBA
:10128000FD0F0906151706F6E9E3E3F3FCEEE6E4C5
:10129000E3FB22352D1C06EFF3FDF4FB090D0E02D6
:1012A000EFEAF5070A04090FFADFDFEA06221C0954
:1012B00002FCE9DDEC081317230EEAEEFBEFE3F87E
:1012C0001A1700FAFC020F181101FD01F7F4060AC3
:1012D000070904F3E2F1101D0CEDE7F50303F5FF38
:1012E00019150001FFEEF5070705030507060E15A2
:1012F0000B030709060503FAEDDFEB080A040A07EA
:10130000FDFF09100F10140D02FBF5F1EFF5FA00C7
:101310000804040D120DFAF20007070B11120D0656
:10132000F6EEFD04FAF9FE040918291AFFF3F0F0AD
:10133000F3F7F900101103050E0A0905F4EDF203A5
:1013400016150D111505F0EEF4FC0407090E191C15
:101350000EF9ECF402040409110F00F6FD0400FC80
:10136000010609080704040904F9F7FF0D14100E1B
:101370000E0900F7F5FCFFF8F50314170D00FBFC50
:10138000FF0300FAFE0F190D0000FFFAF7F4F3FB5C
:10139000071318120A030001030B15170BFE0103B4
:1013A000F8FA050602FAF3F909100E090500FE0124
:1013B000040C1006FEFBFAFDFDFBFE070F0E02FB00
:1013C000F8F90512120B0A0B03040F1304F0E5EBF6
:1013D00003100B060401FAFA040F130F02F7F802C8
:1013E0000B06F6F2FE0A0B0B0B07080906080500B0
:1013F000060D0B06FFFBFD000200FEFE04080709B8
:1014000004F6F1FB060B0C0900F7F5FE0E15130FA1
:101410000C0901FAFE0507050304040505FFFF0595
:10142000070707050403FFFD030909060403030278
:1014300000FEFD0001FDFD0304070D0E070102067D
:101440000500020706030406090906090B05FDFD50
:1014500002060602FCFAFAFE020202050601FE027C
:1014600006060808070707090A0500FF0101FEFC38
:1014700000090D0902FAF8FC01040608080607082D
:10148000080809060200000403FDFCFEFF04040036
:10149000010709090A09090701FDFE0309070100FF
:1014A000030300000307090A0A0903FCFBFB00060B
:1014B00007070600FE0102050A09060300FF0106F0
:1014C00008060504040200030301030502010305E5
:1014D0000404030202010406070907020000FF00DA
:1014E000020305050401FEFDFF03050607050202D0
:1014F00007090605030205070401020302010205AC
:101500000604020102020201000103060601FDFFBA
:1015100004050506070605040202060704FEFCFE94
:1015200001050604040303050501FF01010002048F
:10153000050503020405050401FF02040201040578
:101540000403030405050201010302010200FE0178
:101550000506050402030408080503020202FFFD54
:10156000FDFE000001030507040103080907060545
:10157000040201030402000000020301000103044D
:101580000507050301000103030404030304020229
:101590000304030303020203040402030302010120
:1015A0000202020304050401FF0103040606070505
:1015B000030201010303020202020404020201FF0A
:1015C00000030403020102030202030405060502EC
:1015D0000100FF00010405040200FFFF00010304F5
:1015E00003010000010203030201000101020203E2
:1015F000030201FF000202020302020203030202CD
:1016000002020202030302020201010101010000C1
:1016100000020200FFFF00020202020203040303B1
:1016200002010101010101010102030202020202A1
:10163000030302020203020101020202010201008D
:10164000010202010202010102020302010103037D
:10165000020101020202020202020100000203036F
:10166000020100000100FFFF00020202020202016B
:101670000101010101010101020102030302020152
:101680000000010202010102010102020100000149
:10169000010101000001010101010000010101023D
:1016A0000201FFFE00020303030303020101000025
:1016B000000102020200FFFF000000000000000025
:1016C000000000000000000000000000000000001A
:1016D00000000000000000000000000000FFFF000C
:1016E000FF00FFFFFEDCA292C6296F623116D7AE63
:1016F0001F7E71622BB6828A8A92A6FC4A64742687
:10170000C40676761BB9ABA39AF017ED196375760C
:10171000736E6249301E04EDD9A7848B878B988D38
:10172000888C9BA2B0DED9CCF21C436B79776A6BB4
:1017300079665A737123E0D8BFCBFFF8F831696A34
:10174000554E402C1AF7CBB092858A888889878CB1
:101750008C93BBD5E70714273F483D2608EF0A4284
:101760004D506E797574716E6B695B442DFFDBDCD7
:10177000CDA894888D978B868B8F8F9EAFC2D4BE59
:10178000B0C5D7F211242E2E333D4152523534418B
:101790004849526F76716C6059514B3D1D0604FDEE
:1017A000EFE3D5B28E888988898988898B8C9FB927
:1017B000C3D0CBCDF81825394048534235434C5A55
:1017C00071706669706F675D472A1000EEDAC8B7FE
:1017D000B1B1B7B9B5BCBFB4B5BEC1C5B5A3AAAAAE
:1017E000ABBBCBD1D9E7F71027323C464A454C5525
:1017F0004A4E5A5F6A6B6D6C5A4E3A261E1302EBC4
:10180000E2E5DAC7B8B0B0AEA69B9CA19697ABB1A3
:10181000AEBCC1BDC8DDEC02243635353C4D585C4C
:1018200057433A42485B6555534D3F413C29190B9C
:10183000FCF3EBE2D7CCBEB4B3AAA6B0AFACACA27B
:10184000A2A7ACB2AFB8CEDEEEFE13232B3B4642CE
:101850003F4B5657555052585752525A584D40299F
:101860001B1806EFE1CCBAB1AEBDBFB2B2B0A7A6AD
:10187000B3BDB9B2B4B6B4C4E4F1EEF3FD0C1F319C
:1018800036353E424751575D5D56494349494442CA
:101890003E33292114FFEEE9E3D6CCC4B7BAC3B86E
:1018A000AAAAA397989FA8B6C0BCC0D8EBF7091EF8
:1018B000252532413C3A48483C3D4546454A53552A
:1018C000564E3B3635261101F5EEE5D7CEC8C7C3D7
:1018D000B9BCC7C5BFBFBBB7BCBAB0B0BBC6D0DB15
:1018E000E3E9F80C1D2B363F44474A45403D383A62
:1018F0003F4249504B42382D25251E0D01F8EADDA7
:10190000D8D4D2D1CBC4BFB9B6B4ADA8A6AAB3BC03
:10191000C2CBD5DBE9FD050A1A262B333D414346F0
:10192000423F43474A4947474041413224170D0946
:1019300000F6EADEDAD8CFC2C0C1C2C3C0BDB9B2B8
:10194000B2B3AFB2BECCD8E3EE0010111A292C30DE
:101950003635353C403F3A393F414446403B3327DA
:101960001F140A01FCF9F2EBE5E3E4E1D8CCCAD09C
:10197000D1C7BDBAB7B7BBC1C5C7CEDBE1E7F4017C
:10198000070C151E29303133373B3B373836353E8F
:101990003E37332D2D302C1D0F0F0E09FEEEE6E2E3
:1019A000DBD0C8C8C9C2BAB6B4B5B6B3B1B8C2CD37
:1019B000D5DCEAFA0510171D2831312E2F313334CA
:1019C0003738383B3E3E3932302D2317120E05048E
:1019D0000602F9EFE5E1DACEC9CACAC9C5C1C1C07C
:1019E000C3C5C6CCCECFDAE2E5EFF9FE070E121A78
:1019F000242E333130353A3C3E4245433E3735386C
:101A000030241C160D05FFF5ECE9E3DBD6D0CDCC78
:101A1000C3B6B4B9B8B5B7BEC8CFD4D9DFE5EEF612
:101A2000FD071521252930363B3B3735373736370B
:101A300037332E2B2421241F140B0604FBF3F0ED67
:101A4000EAE5DBD3D1D0CCC9CACAC5C3C7CCD4D987
:101A5000DAD8D9DDE2EBF3F7FC060F18222A303191
:101A6000303438393C3C3937363533322E29221B55
:101A70001107FFF6ECE7E2DFDBD4CFCBCBCDCAC753
:101A8000C6C5C4C5CBD3D8D8D8DDE3EDF9FF000770
:101A9000131B21292F3234363938343333322D2673
:101AA00024241D191814120F0902FAF6F6F4EFE8AF
:101AB000DED8D5D1CECCCAC7C5C4C8CDD0D6D9DB27
:101AC000DDE1EAF6FE01040B111B262C2F3131302B
:101AD0002F313536343230302F2E281F160F0B069B
:101AE000FFF8F0E9E4E1E0DAD2CDCDCED0D3D2CF29
:101AF000CDCDD0D6DDE3E3E3E9F2FD040402040A30
:101B0000141E25292B2C2C2C2C2F302D2B28211E5C
:101B10001A141010111314120A0400FCF7EEE3DA81
:101B2000DBDBD8D4D0CCCBC8C6CACFD5DBDCDBDD81
:101B3000E2EBF4FB01070E171D2024272728282994
:101B40002D2E2E31322D292A2924211D181109026A
:101B5000FBF5EFE6E0DEDCD9D7D7D7D7D6D5D4D39F
:101B6000D1D5D9DCE0E3E5E8EEF6FF00FF0003099C
:101B7000141D1C191C2225272A2C2E302D2A29241D
:101B80001F1D17101013110B05FFFBF7F3EBE5E218
:101B9000DFDDDBDAD7D4D2CECCD1D6D7D7D5D7DBE1
:101BA000E1EBF2F8FE040D171E2226262425272736
:101BB00027292A292626282824232019120B060340
:101BC00001FBF4EFEBE9E7E4E1DDDAD9D8D9D8D7C6
:101BD000D7DADDE0E3E6E6E8ECF0F4F6F7FAFE0447
:101BE0000B0F14181B1E2227292B2C2C2B272324E8
:101BF000221A1515120D0A0B0A070400FBF8F7F25A
:101C0000ECE7E1DDDBD7D4D0CCCCCED1D7DCDDDF47
:101C1000E2E4EAF1F7FB010810161B1E2122232340
:101C20002427272524232223221E1A171513100DDB
:101C300009070500FAF6F2F0EDE7E2DFDEDDDAD7BC
:101C4000D6D7D9DCE0E2E4E5E9EBECEEF0F2F5F72B
:101C5000FA030D1113151A1F21222325292A241FE7
:101C6000201E1B1A1813121211100C09060400FB77
:101C7000F7F3EEE9E5E1DCDADAD8D6D5D4D5D8DB6E
:101C8000DEE0E1E3E7ECF2F9FE03070C12181D1F9A
:101C9000212122242523201E1E1E1D1C1B19171561
:101CA0001312110E080402FDF7F5F2EEEAE4DFDD8F
:101CB000DDDBD8D7D8DBDEE1E3E7EBECECEEF0F2EE
:101CC000F2F4F6FA01070B0E11151B20232323242F
:101CD000252423221F1C1916151414120D0907059B
:101CE00002FDF8F7F4F0ECE8E5E3E1DEDAD9DBDB5E
:101CF000DBDDDFE0E2E3E5E9ECEDF0F6FB01070C0C
:101D00001014171A1D212121222221201E1D1C1C06
:101D10001B17151515120D0A0602FFFDFAF5F1EE57
:101D2000ECE7E3E1DFDDDCDDDEE0E1E2E5E6E7EA8A
:101D3000ECECEDEEF1F5F8FAFD00060C11161C21A5
:101D4000242524252726221C19161514110F1111DC
:101D50000E0B09070501FEFBF7F2EFEBE7E4E1DF0D
:101D6000DDDCDCDCDDDFE0E1E3E6E9EBEDEFF1F526
:101D7000F9FD01060A0E13181B1D1E2021201F202D
:101D80001F1D1B1A19191613120F0E0C080503013B
:101D9000FCF7F3F0EDEBE9E6E4E3E2E1E0E0DFE0BD
:101DA000E0E2E5E8EAEBEDF0F3F6F8FAFD01060C07
:101DB000111315191C1E1F2022221F1D1C1B181376
:101DC0000F0D0D0D0E0E0C0A080400FCFAF8F4EECF
:101DD000ECEBE7E4E2E0DFDFDFDFE0E1E3E5E6E8CC
:101DE000EBEFF2F5F8FD0103060A0D0F12131519BA
:101DF0001D1E1E1D1D1D1C1A1817161512100E0D66
:101E00000B09080501FEFBF8F3EEECEBE9E6E3E174
:101E1000E2E3E3E3E3E3E4E5E7EAEEEFF1F3F7FA25
:101E2000FCFF010305080B0F14181A1D1F1F2020AB
:101E30001E1C191714110E0B0B0C0B0908070603B7
:101E400000FDFAF8F4EFEAE7E6E5E5E4E3E2E2E2D2
:101E5000E3E5E7E9ECEDEFF2F5F8FAFDFE00030744
:101E60000A0E12141517191B1C1B1B1B1B1A181703
:101E7000141110100E0C0A09070400FCFAF7F3EE17
:101E8000ECEBEBE9E7E6E5E5E5E4E4E5E8E9EAECD7
:101E9000EEF0F2F3F5F7FAFCFF02060B0E10131644
:101EA000191A1C1C1D1E1E1B191713110E0D0B0ACF
:101EB00007070706040301FDF9F6F4F2EDEBE9E884
:101EC000E7E7E6E5E5E6E7E9EAEBECEEF0F2F4F663
:101ED000F8F9FBFD01060A0B0C0F111417191B1D55
:101EE0001D1B191816151311100D0C0B0B0A0804E5
:101EF00001FEFCF9F7F5F3F1F0EDEAE9E7E7E7E6D3
:101F0000E6E7E7E8E9EAEBEEF0F1F4F8FCFF0102BE
:101F10000406090B0C0F1316191B1C1D1C1A18168E
:101F20001411100E0B0907070606050401FFFDFB3F
:101F3000F9F8F4EFECEAE9E8E8E7E7E8E9E9E9EBE2
:101F4000ECEFF1F3F3F4F6F8FAFD00010204070BED
:101F50000F1213141618191A1B1A181513100E0D38
:101F60000B0A0807050505050301FEFCF9F4F0EE70
:101F7000EDECEAEAEAEAE8E7E7E8E9E9EAEBEEF1BC
:101F8000F4F6F8FAFCFE0002060A0D0E0F10121508
:101F9000161616171818171614100D0B0A08070630
:101FA000050404040200FDFAF7F4F1EFEEECEBEAAD
:101FB000EAEAEAEBEBECEDEDEEF0F1F3F5F6F8F929
:101FC000FBFDFF02050708090B0E11141516171665
:101FD0001717161412100F0D0B080605050504033C
:101FE00001FFFDFBF9F6F4F2F0EDECECEAE9E9EAC9
:101FF000EBECECEDEEEEF0F2F3F4F6F9FBFE01049F
:102000000607090B0D1012141517171716151412C1
:10201000100F0D0C09070707070502FFFFFEFDFB68
:10202000FAF7F4F1EEEDEDEDEBEAEBECEDEEEFF0BF
:10203000F1F2F2F4F5F6F7FAFCFDFE0103050608ED
:102040000B0E10111213151617161512100F0D0D79
:102050000B0705040505040200FFFEFCF9F6F5F484
:10206000F2F1F0EFEEEDECECEDEDECECEDEEF0F28C
:10207000F3F5F7F9FBFD00020406090C0D0D0E1037
:102080001213151616151311100F0D0B0806050463
:102090000405040200FFFEFCFAF9F6F4F2F1F0F098
:1020A000EFEDEDEDEEEFEFEFEFF1F3F4F6F7F9FA18
:1020B000FCFDFF0102040506080A0D0E10111212A4
:1020C00013121211100E0D0B0A0907050303020368
:1020D00003020200FEFBF8F6F4F2F0EFEFEFEFEF91
:1020E000F0F0EFEFEFF0F1F2F3F4F6F8FAFCFDFFA9
:1020F000020305070A0B0C0D0F1011111212121218
:10210000110F0E0C0A07060505040302010000FF6B
:10211000FEFCF9F6F4F3F2F2F1F0EFEFEFF0F0F18C
:10212000F1F1F2F3F5F6F7FAFCFDFEFF010203050B
:102130000708090A0B0C0D0F10101010100F0D0CD2
:102140000B0907060505050403020100FEFDFBF966
:10215000F8F7F6F4F3F2F1F0F0EFEFF0F1F2F3F359
:10216000F4F4F5F7F8F9FBFCFE0002040507090A90
:102170000B0C0D0F10111211110F0D0C0B0A09078A
:1021800005050403030301FFFDFDFCFBFAF8F6F56A
:10219000F3F2F1F0EFEFF0F0F1F3F3F4F5F6F6F817
:1021A000F9FBFDFEFF00000103040506080A0B0D04
:1021B0000E0F10100F0E0D0C0C0B0A080605040371
:1021C0000302010000FFFEFDFCFBF9F7F5F5F5F455
:1021D000F3F2F2F1F2F1F1F1F1F3F4F6F7F8F9FBC1
:1021E000FDFEFF000102030507090B0C0D0F101186
:1021F00011100F0E0C0B0A0A080605040302020256
:102200000100FEFDFCFAF9F8F5F4F3F4F4F4F3F34D
:10221000F2F1F1F2F2F3F4F4F6F8FAFBFCFDFF0050
:1022200002030405060709090A0B0C0D0E0E0E0E1B
:102230000D0C0B0A0807050404040302010000004A
:10224000FFFEFCFAF9F8F7F7F6F4F3F3F3F3F3F320
:10225000F2F3F3F4F5F7F7F8F9FAFCFDFF010102E8
:1022600003050607080A0B0C0E0F10100F0E0D0BBE
:102270000A0807050504030303020100FFFEFDFC35
:10228000FBF9F8F7F6F5F4F4F3F2F2F3F3F3F3F401
:10229000F5F5F6F7F9FBFDFEFF0102030304050661
:1022A000070708090A0C0C0D0D0C0C0B0A0908078E
:1022B000050404030201010000FFFFFEFDFCFBFA20
:1022C000F9F8F7F6F5F4F4F4F3F3F4F4F5F5F6F8B9
:1022D000F9FAFAFBFCFDFEFFFF0001030405070805
:1022E000090A0C0D0D0D0C0C0B0B0A090706050451
:1022F00004040403020100FEFCFBFBFAF9F8F6F605
:10230000F6F6F6F5F5F5F4F4F4F5F5F5F6F8F9FB6F
:10231000FCFDFEFF000000000000000000000000C7
:10232000000000000000000000000000000000FFAE
:10233000FFFFFFFE03FA092AFDDC01F4EC09F8EACD
:10234000D0D6FEEBED1A0EECED1014FB1B04F5F8E5
:102350000233221F38120211FF0100E9EFD6BCE858
:10236000E9E4FFF2E2F603F40A1E2422190F2334F3
:102370001106230FF301EEF5EACCD7DCC9BED8F87D
:102380001404FE1F09072818FD00FC0B350CD3E6CA
:10239000F2DEF7EDEA120EF8E7F11518010E10FF64
:1023A000052D25F6FEDDE21313F8E9DCCE1E0FE75E
:1023B0003F32000BE9E70B01DBF503F80F04162AA7
:1023C000E9DA0BF3F620F6E2E8E80B03022005F366
:1023D0000817FDE1F9040CFBFF0A06FCF3FF0905F1
:1023E000060F1320F8E6F7030D090C1F18F4F5FB90
:1023F000EEF805E9FA16EEE3FEFEF41914F4000710
:102400001B0BF20907F5121EF8F7F9CCEBF3CB0220
:102410001CECF5FADC131E052B1102220EF704F951
:10242000E3F204FDF5F70815EDEB152401182DF482
:10243000F505FCFAECDCEAF8F30213EFDB141DED12
:1024400004292A1AF70000F502FAF0EAFC00F5EB7D
:10245000F1F8FF0E2218011C25F8F701DFE9FAEF69
:102460000209FF040B00F3031622FBF407FAFD0434
:10247000F4E6FCF5FB1FF5E10D01EAF60D1502127D
:102480000EF3FF090E12E6E10A00FAFBFEFFF2F37B
:102490000B04143413FF01F3030AE3E8F3EE031112
:1024A00008FCFD0706F80906F5121EFFEDFBF6EE27
:1024B000FDFFF40E120402E9EB00FBE1F6120C083A
:1024C000080802F5011503EFFA130CF6F700F5E121
:1024D000070D00070701D3EB16FCFBFDF7FF030E0A
:1024E0001AFFE3010AFC0D04E3F4010108FE0E0EDD
:1024F000E0FB2A0A090AEAF6E5F6300EE6F0F100FA
:10250000071419F6F80DFBF610FCFCF4E5111202A5
:102510000F01ECEB011C05F509FDEA091301010AA5
:1025200011FCF00502F5EBDDECF3F7181BEDFE1BDB
:10253000F205241004F6F601E6E812FAEAFFFD0FB0
:1025400013F1F904ED0212051412FEFE030507FB58
:10255000FE05E8F70DF8F0F0EC060EFC132204F28D
:10256000FE03FE060BF5F204FAF607F8EFFC040989
:10257000080803FEF9F5F4000AF8FB08EFF908E98A
:10258000F20C01FE100BFF01FDFD020BFEF7FEF247
:10259000F6FEF5FA020403080902F90301F101103D
:1025A00003FDFDFAFDFEFFF9F8F2F4080EFA05113D
:1025B000FA08120305FBF4FCF8FB06F3F201FD0434
:1025C00004FB0602F90B0D00080FFFF7F903FCF1FD
:1025D000FFFEF1FE01FC02FA020800050B0C03F9F4
:1025E000070AF5FB01F0F40001FDFEFE01FD020DFE
:1025F00004FE0308FCF2FD0801F4FE09FBFD0905D9
:10260000F3F20201010501FD01050805F70309F5D3
:10261000F903FFF8F40406F40411FCF50703FFFEC8
:10262000FB03FAF70503F7FC0A06FAFE0700F6FDBE
:1026300002FBFAFD0803FC060703FCFBFEF7FD0A9C
:1026400001F4FC0802F8FF0905FE0601F3F2FC059F
:10265000F8F80902FA0704F9FD0403F7FA0502FB8A
:10266000FB0001FDFF0801F4FD0601FE0104FD026F
:1026700007FFF9FC04FDFAFE0102FD01000000085D
:102680000DFEFB0703FBFBFBF5F90000FFFD040457
:102690000104030600FC03FFF90004FEFBF900003F
:1026A000F80302F50003FE04030408FFF90301FE2A
:1026B0000300FBF6F80102FDFE0000050600FC0425
:1026C00004FAFF00FE02F9FB04FCFE0905FDFBFE17
:1026D00003FFFD03FDFB04020000FFFFFBFAFF0404
:1026E000FFFD0304FDFF07FFFB0203FEFEFEFDFCF2
:1026F000FAFEFFFE020302010203FEFD0201FBFAE5
:102700000000F9FE03FEFD030603FEFE01FEF9FED6
:102710000301000302FDFE0000FCFD01FEFD0201BD
:10272000FCFF010100FF0202FCFDFFFBFD010300B5
:10273000FD0204FDFDFFFEFEFE0102FEFE02FEFCA8
:10274000000202FFFF0200FC00FEFAFD010300FF91
:102750000201FD0003FFFE0001FEFE00FFFEFF017F
:10276000FFFF0100FEFD0002FCFE020300FD01026E
:10277000FFFE00FEFCFFFFFF00FE0001FEFF020067
:10278000FF01FFFDFFFF01FDFD0301FD010200FF51
:10279000FDFFFFFD0000FFFFFF0000FF0201FE0242
:1027A00003FFFF0000FEFDFF01FFFF01FFFE000031
:1027B00000FFFF0100FF0101FEFE0000FFFF01FF1F
:1027C000FEFFFEFEFFFF0100000201FF0000FFFF11
:1027D000FF0100FEFFFFFFFEFF00FF000100000001
:1027E0000000FFFF0000FFFFFF00FFFF00FFFFFFF3
:1027F000FF00FFFFFFFFFF000000000000FFFE00E2
:1028000000FEFFFFFFFF00FFFFFFFF0000000000D2
:10281000FFFFFFFFFFFF00FFFF000000FFFEFFFFC5
:10282000FF0000FFFFFFFFFF0000FFFFFFFFFFFFB4
:1028300000FFFFFF0000000000FFFFFF000000009E
:1028400000FFFF00FFFF00FFFF00FF00FFFF00FF92
:10285000FF0000FF00FF0000FF00FFFEFFFFFFFF83
:1028600000FFFFFF0000000000FF00FFFF00FFFF70
:1028700000FF0000FFFF000000000000000000FF5C
:102880000000FF00000000FFFFFF00FF000000004D
:10289000000000FFFF00FFFF00FFFFFFFFFF000041
:1028A00000000000000000FF00FFFFFFFFFFFFFF30
:1028B00000FFFF00FF0000FF000000000000FF001D
:1028C0000000000000000000000000000000000008
:1028D00000000000000000000000000000000000F8
:1028E00000000000000000000000000000000000E8
:1028F00000000000000000000000000000000000D8
:1029000000000000000000000000000000000000C7
:1029100000000000000000000000000000000000B7
:1029200000000000000000000000000000000000A7
:102930000000000000000000000000000000000097
:102940000000000000000000000000000000000087
:102950000000000000000000000000000000000077
:102960000000000000000000000000000000000067
:102970000000000000000000000000000000000057
:102980000000000000000000000000000000000047
:102990000000000000000000000000000000000037
:1029A0000000000000000000000000000000000027
:1029B000000000000000FF0000FE03FA092AFCDC12
:1029C00001F4ED09F7EBD0D6FEEBED1A0EE9EB12B0
:1029D00014FB1C03F4F80333221F37110111FE010D
:1029E00001E8EED5BCE9E8E500F1E1F602F40C1EE1
:1029F0002422180F23331307210EF301EDF5EACC3F
:102A0000D8DCC8BEDBFB1303FE1E08082A18FCFE38
:102A1000FA0C350AD2E8F3DDF7EDEA140EF7E6F228
:102A20001516020F0E00062C23F6FEDCE31313F836
:102A3000E8DBD0200DE84031000BE8E30A02DAF6CB
:102A400002F91003172AE7DA0BF2F720F5E0E7EABC
:102A50000DFEFE2204F20918FBE2FA040CFB000A48
:102A600006FDF3FF0B05020D1521F5E5F6020E0933
:102A70000E2119F4F4FAECF809EAF914ECE4FEFC7E
:102A8000F31B14F502091E0CEF0809F7151FF7F6E2
:102A9000F4CAECEECA051AE8F1F8D7111F07321391
:102AA00002260FF502F7E1F307FEF4F80A14EAEA4A
:102AB0001B29FE1B2DF0F808FAF8E9D6E5F4F3041B
:102AC00015ECDA161BEC052A331FF50503F102FDA0
:102AD000EFE6F801F3E9F5F6F80E2816FF2024F5E5
:102AE000F4F9D8E9F6E8040CFE070AFBF5051C2703
:102AF000F5F205F7FC04F3E0FEF7FD25EBDC10FA38
:102B0000E2EC0E19001809EC01091815DCE20CFBC7
:102B1000F7F7FBFFEBEB0C0520411501FEEF0A0E6A
:102B2000DDE2EFED071B11FCFD0C09F8060D0015A9
:102B30002100EBF7F7F2F9FBF111110706E0E807C6
:102B4000FDDDF515120E0C0C02F50B1F03ECFC1D40
:102B50000CEDF3FDEFE1150DF90D0B00D2F41EFEA7
:102B6000F7EFF402F90C26FAD30615011B0DDDF977
:102B70000AFC05FD1915CFF9340E1108E6F1DAFC4F
:102B8000430DD4E9F9090B1F21EEF511F7F00FF70A
:102B9000FCE6D61C16FE16FBD7DD052F04EF0DEF65
:102BA000E3111807000D1EF4EB13FFECDDC7E3E89B
:102BB000F32D23D4FB28E30A3D1B04E4EBFDD4E70B
:102BC00025EBD4FFFB1A21E6F500D80C2A051B1FC4
:102BD000F7FF0F090DF3FB04CFF518F4EDE5DC1654
:102BE0001CF7243501EDFD03FE101CE7E309F3FBA0
:102BF00015EAD6F50F1614100806F3E2E5051AEAF1
:102C0000F814D7F612CFEF1AF9021E0A0B07F4FEDA
:102C10000917F7EDFADFEFFCECF80A0C0B110CFAD0
:102C2000F615FADA052307F9F7F0F1FC01EAEDDF12
:102C3000E4111EF3001AF21E32090BF9E5F2EDFC65
:102C400011E6EB04F90B09FD0CF4F12A2904112417
:102C5000FEEAFE11EDD704FAD8F6F8F906EC0C1BE3
:102C60000416202405E61319DBF002DBE2FF08F767
:102C7000F9F904F700220CFC0F18F2D9F51AFED46A
:102C8000FE17EFFD1E0FD3D20C05061403F7051235
:102C90001806DE0E14D6ED16FDE2E61208E51B332B
:102CA000E8DF1E0CFFF7EE0EF4EC1509DEF62D162C
:102CB000E5FE21FAD7F708F0EEF917FCF31C200E19
:102CC000EDEDF3E0FD23FDD7F62206DFFF2717FD2C
:102CD0000F01D2CDFC1BE9EF2D07F01F0AEEFF100C
:102CE0000DDCEE1B02DFF10204F2012EFCCBF00939
:102CF0000BFBFC0DF21228F7DEF70DF6F6F3080ECB
:102D0000F70C0302072637F1ED2705E5F3EBD8F1C1
:102D1000FBFF01EB12160F12112BFBF016F5DAFF79
:102D200011F6E9E606F4D71C09D0130EF81F141AA1
:102D30002FF0D91D05FD18F8EBC9D10B0EF7FCFFDC
:102D40000A2C2A00F0240DD6FCFBFB11D6EE17E26C
:102D5000013714E9D7F51CF4F117ECED230D080643
:102D6000FCFDE5DAFF25F5E91E22ECFF35F2DE1960
:102D700013F2F7F0F2E8D4F8FDF20514100E18186B
:102D8000FBF9160BDCD60B06CCFB20E9EC1F30154B
:102D9000F3F60CF6D9001C08041C10EFFC0101EB43
:102DA000F413F5EE1F06DB01160E03FA2020E2ED08
:102DB000F3DAEB122BFEEA2227EBEAFCF3F4F40E33
:102DC00021F6FB24EBD90D261BF9FE25F9DF09E9D5
:102DD000CBE4192803051D0FE2102FF3EE0C0DEDC7
:102DE000E804FAEA060DF3F7100CF1DC1624DAFA1F
:102DF0002C31FDE21E23F5EE0FE3CCF9F60100EADB
:102E00001312E90B21FC041EF4E4F20519E2EB3B7A
:102E10000FDE191F00F1DF01F8DD0BFDEEF9F812EE
:102E2000F7F43515E63730E9FB05FDDECD0311E794
:102E3000F51AF6E9081205EE022600F62D11D9E47E
:102E40000A14EEFE1FE8DAF8E7F1ECF3240E12366E
:102E500016F90614FAE6FB19F7D5EDF4EEE5020AC9
:102E6000E8061F12150B0309FAF90C03FAF3F50132
:102E7000E5FD13EDFDF4F61AF9EAF8E9F81B1B1D60
:102E80001F020EFDD90706E7F1F9FB040AFB01F268
:102E9000F20B0C1A1A0F03EBFA05E8000DE8F6180E
:102EA0000F0EFAE1FAF0EA161907FD0007050C14F7
:102EB00002F902FDF5FE02DBD6F1FF1414161BFC2D
:102EC000EE000B110F00FFEBFA19DDD504E0022430
:102ED000002601E20DEDED21161014F7130BDB13A4
:102EE00000CEF5FCF0F90DFDF7000C250D1917F6D5
:102EF00002EADDF9DEE70CEB0E2FF7F70B061AFC02
:102F00000026F0FB0CE2F7FFECFC00F7FDF0DCEF35
:102F100000EF06181E2C010923F3FD15DFF0FDC795
:102F2000E4F6C9EA04122B0210160C1CFCF804FA91
:102F3000F3F7F9FDE1DB09F5E80CF4001AEB1031C9
:102F4000040E29F3EF24F9ECF6E5EADEE705F0E7F5
:102F5000FB0D1F191B271F030205EDF5FAE9DDFB29
:102F6000FEE9EE0304EC1525082116F9250BEA000D
:102F7000F6ED0A01E3F3F0F2FEE9FB170D0AFE0598
:102F8000211413280EEB0401E6DFE0E2E90503FC5F
:102F90000911130EE7001B01090805EAEE07EFF31C
:102FA000F2EDE5FB11060F0C14120621191B08E4C3
:102FB00003F2F00AE3C8E9E6EA1701051A0F2A2925
:102FC000080BF8F1FFFBF4EEEEE9FCDCE710FDFC8A
:102FD000F2050D0D240BE80A160603F1F2F5E3F8ED
:102FE000F8D302110A2407040DDEFE23F3FE03DCEE
:102FF000D3E9FB070F0607F3153112FEEEE7010BCD
:10300000081302DFE0FBFFFF0E1BF0E5220B042696
:1030100003E3FA110A1804E6E6D3F217FFF9F6FA09
:10302000F5F914181506140DFE221BEFEDF1D9FE6B
:1030300005DEF4EFD9101F0C0D1618F3141D09143A
:103040000DEEDDFF02F3FCF0D4D6F8120C030507F9
:103050000416160F270BFE02DAFE08CD01F7C0F3A7
:10306000000603F81D1CFB1C28FD0601E5E8F5F928
:10307000FFF6EAF0FBE7F417F1EE0A0F241D181231
:10308000F6E9F5F6FF0BFCE0D9E9F3FD12230D0399
:103090000E3108E805F6E7031AF5F302DFE301F362
:1030A00004161419F8F407FFFCF6E40E190C13EEDD
:1030B000E3EBE9FF0B0518FCECFDEA082C01F81620
:1030C000F1021BE0E3FEEA03230CF7F206FFEB0636
:1030D0000BFB0CFEE7FB06FAE3F1FFE92146FDFAE4
:1030E000FBD8FB04F902F7F51312F4F90F26FF00E1
:1030F00021EFDFF7F1E0F60B03030BF3FD1E04F302
:103100001B0CE41E0ADF0A0BEFF8FCFFFEF611FEB3
:10311000E906F0F20AEB00290A011A0FF30C1DF17F
:10312000DCFE00EC050CED000DED07FED6FD05FD07
:103130001C140E0CFC1802E62004D000F2CDF3049F
:10314000F3EB0911182B0A070FE2E81D12FF120911
:10315000EDE9F5F6F0001405FC0CFDDFECFBF215D3
:103160001BFD11FAEB03FAECFE12FC0508FF040448
:103170001400F70E1005F6E5E3EEE5F20D07051F66
:103180001B010207EBF5290D012208DDD6DDDAFA75
:103190001108030A1002F3000CFC011E1301FFEFDB
:1031A000FAEFDB0112FE140DDCEAFFF6F81009114C
:1031B0001E0C09EAE6F3F4060C040BF1E205EFE657
:1031C000271FEC00110FF2F00FE2E8130F060204C4
:1031D000F9F6F7020CF9141FF2F80FFCE2EAEAFE26
:1031E000020B2EEEE32505FB18FF040CF2030BDEA9
:1031F000EB0EF2E9F81009F80D09E8FA12FDFC03EC
:1032000010120312FEE209FFDF03FCF309E7F411D9
:10321000EB0325040412110B0007F5E0F2ECEA0AB7
:1032200008F7000CFEE90E22050C06ECFDFCF1038C
:10323000FBE71618F505F2F6FCEC01120F1C1CF763
:10324000F9FEE8F602F0EBF9080504FAFA10F2FAD2
:10325000260F050D09EDF00503FEF0FBF9F7FDFB68
:10326000FBFB0411100A030C08F3F905FFFB00F542
:10327000E4EEFFF8F5F90D170B1B2004F801F9F740
:10328000F1FB01F9F7FEF4E203FAF90E04F809097B
:103290000110F90A09FC1808F90AEFEF09EBF1FF30
:1032A000F50305FE11FFF819070B160008FAE403F1
:1032B000FFDEFC02EA0D01F213000010F9F812FE25
:1032C000FB0EEA010CF3F9F6F6FEF3F21004F50C2E
:1032D00013FE06020507F3FBF4F3FEFF0405EFF906
:1032E000FADF061AF80E2601F80804FAF7FF00FEC6
:1032F00000FE04FFF3F0EFFBFD010A0B080B0A02CE
:103300001004EFFA08FBF7F9EEF3060CF60B11FBCD
:10331000FA00F1EC0AF7FD09001407FF110BFBF9A5
:10332000060CF2E2FBFED5F11E00020B07FDF90BC5
:103330000CFEFC11110CFCFAFFE1EC10FF0D0EFC71
:1033400002E6F2F9EA0009F610261619F9F204E885
:10335000F00CF7F3F3F90AFBFF00FB0E1300130D5B
:10336000EEFEEEE20613050B02F5F2EC0001F80D9D
:1033700001F31A03DF0B0AFB12100D0CFBF5E7F14A
:10338000FCF0FD03F7FE0EFE0000FC05091401FF32
:103390000BF5E9FDF8EC0215FFFF05EBF8FAEBF48D
:1033A0000B0514280B03FD040DEFF0F8F00B04EBF4
:1033B000FBFBF2020C06FFECFA08F5010702121102
:1033C00005FDFD10FAE1EE090FFB0904E3E40A0133
:1033D00002160B0A070101FDF3FAEFF0F40B19F8DE
:1033E000030EFBEC04150F0BFB06FEE7F4F6DFF90A
:1033F0000F0B0C050E00E3FB13FCFF1F0BFCFEFD87
:10340000F4E9FFFDEEFB0E0AF4F6F1F805FF151ED8
:103410001B0A0303ECF50DF6EDFAEAF2FBEEF807F2
:10342000F90A1E141C0D04F3EF00F7F3100EE5FB70
:103430000CE8EC09FBF9061009F6F8F0EC010005C0
:103440002E1DFD0FF9E6F7EDF3FAF806FEFF09F37E
:10345000F204FA0719FF051200FE02F6FF06F4EE69
:10346000040CE5F206F3FB0F0E00FAFC07FA00115C
:10347000091B13F80D05EFEFD7F40CF6F105FFE289
:10348000F60501041012010A1304F70609EC0706F9
:10349000F411F5E6F9F3EFFE090000030D01071E34
:1034A000FF051DECF01D00E2F3F9EDF6FDF907074D
:1034B000FE0208040307080C00090BF60A04E4FCEA
:1034C00001E4F9FCD6F316FBFC1B0E1C270503FBDD
:1034D000F8F1F1FEF6F2F5FCF7F5F90306FF120537
:1034E000FE19FBFE0EDE0119ED0C13F7FCF5E6FBF1
:1034F000F4E30A07020A071601000B080C0304FD97
:1035000004F9E8EEEFF1EEFB06020D05FC1918FDDB
:103510000113FEF90BECFCFEE90904EAF703F4F0F1
:10352000F2FB02FF2228FC0619F3EC0BFEE8FE0773
:10353000F7FBF3F2FAE9EB060D0914210FFB0F0E6E
:10354000F2F402F9EAF6FEECF403F9FD0BFF0711C1
:10355000F9060CFB010907FF0BFEF1FDF6E8F80583
:10356000FAFEF5FA0CFF0808EE1618F21217F4FF2F
:103570000EFBF6EDF20DF0F30C04FFF50D02F70271
:10358000FAF2F51306F406131D060C1BFDF1F0E923
:10359000E9E6E6FFFCF3120E0110090D0DFC160D15
:1035A000F508F6E0F4F8F606F6060DEDF600F0EC98
:1035B000FAFE130D0E2D1C1609F3FDF4EFF9EBD9ED
:1035C000F1F6EAF80612070A2814051101F6F7FDCC
:1035D00002FEF8F803F3F706F1F0FC03F2F4100F23
:1035E0000806150F0A160903ECEEEBE0EBE9FC0305
:1035F000F7091F06FB130701120300F9EAFBFBF5AD
:10360000FC0507F5FB06FBE9FC02F6FF111E0112A3
:103610001CE8F504F4F9F0E80704F10B05FC020DD1
:103620000DFAFF1700EC0103ECE8FE04030D150C86
:10363000FCFF0A01EAF3FAF3F0FD1BFEF918100291
:10364000FE0C03F3F1FEFCEA0309F9F5F90900FEAB
:103650000F0BF4EF0E0D010F0903F30013F5F1FB4F
:10366000F8F4EFF0FAFAF9140601290F0606F40B44
:1036700006F20002EBE9EDF4FDF0090BF0131C007B
:10368000040D06F6F5140DFC0500F9F1EAEFFAF069
:10369000F10200FA101D08100E0606FFFDFDF6F0FF
:1036A000FAFD0301FA01F3F602FEF2F41000FF2125
:1036B0001001110BFBFAF9F8F9EBEEF4EDF7F50652
:1036C00014FE0A1B1601060BF1FE02F5F3F6FDF1DE
:1036D000F903FCF4FA0801FF031204FA1C14FF06B4
:1036E0000102F1E501F7DDEEF5EB080E0A120F1EFF
:1036F00011080D0200EEE4F3F9FE03F8F501F409F8
:1037000010EF0606F90F130A07060200EDFC0BED99
:10371000EEFBEFFAFFF50505F70D1E0A090E06FB95
:10372000F00003F4F7F8F1F4050806F6F905FD02D8
:10373000040B02F70F1204070DF7ED00FCF2F0F690
:10374000F4F1FF03090B030B0D08090D08F4F3F462
:10375000F2FAF805FDF3060D020302F904F6FF0E76
:10376000F6FD10FCFF110800F3FE03EEF1FDF7F487
:10377000FB080F01030E0903FF0B02FA00FAF8FE23
:103780000503F6F4FFFAFC0AFCFDFBF90E04F4094C
:103790000BFB081603FB00F6F6F7FAF6F2F9FDFA52
:1037A000FB090A0910060803F5FEFFF8FC020305F1
:1037B00002FEFAF2F4F3F400FD0411050B0DFFFE16
:1037C0000703FE01FF00F2F400F1F10805FE0AFF15
:1037D000F708FF040CF90B0DFD0300F8FCFDF903DD
:1037E000F5F901F0F8F9FE0F07091408050BFCF8CC
:1037F000FFF70200F304F9EBFDF5EA070AFE0CFE01
:103800000413FC000B07080B090DF6E2FAF1E7F7C9
:10381000F40000FC0906010112030016110603035F
:10382000F7EFF9FCF5F401FAE9FAFF0109060807D8
:103830000D0B1009F7FE06FAF6FEFAEBEAFFFCF6AE
:103840000306FF0705060F0002070302070E02F535
:10385000F5F4EEF5F9F3F90403000F07F3070D0093
:103860001A11FB0700FBF7F1F5F1EA0001F7110F60
:10387000FAFC0100FEFEFF040401130AF80405F03F
:10388000EEFCFDFFEFFB02F1080F0304070B0E0136
:103890000405EFF0FEFAFCF9F9FEF20107FF090A50
:1038A000070201FE0500F905FFFF0BFEFD00F8FD14
:1038B000FDF5FF02F10301F91703F60F08FE0107FA
:1038C00001F4F705FAF00405FAFE0602F5FC03FF21
:1038D00005040400FF0607FAF60608F7FD0EF5F2E8
:1038E00006F8FCFFF703FFFD0A06FF03040002FFD2
:1038F0000302F80301F6FA05FFF304FAF00B0400E3
:103900000F070004FDFE06EEFA0BFBFFFF00FEF9B9
:10391000FAFAFC0102FD050D03FB000900FB05009E
:10392000FC0206FFFBF9F700FEF7FE00FB020BFFAF
:10393000FB0903FF0502FEFDFE01FEFCFAFBFD078D
:10394000FEF907FBFE04F8010A000204FC0405FC72
:103950000405FBF9F9FFFDF9FE02FAFD0D04FEFC7A
:10396000000200070702FCFAFA0000F0FAFBF70A6F
:10397000FEFA0802FE03FEFC06020B0BFD0A03F42E
:1039800000FFF9FE040402F6F306FEF704FEFE0350
:10399000080C04FF04FEFC03FAFFFFFA02FCFA0322
:1039A000FAF9FDF70603F90C03F609FFF506FF0027
:1039B00001FB0303FDFCFBFAF8FE0700FAFF00061B
:1039C000040005F8040AFDFFFFFAF6FF03FEF5FB0D
:1039D00004FE03FEFE05FB000A000506FDF8F8FDE7
:1039E000FE00030C01FC07FEFA0204FCFA0805FACB
:1039F000FBFCF3F7080503020004F8FC03F80008D9
:103A0000FB0710F90004F7FEFDF90606FB0001F9BB
:103A1000F9000103FF060CFFFF02F9FB060304088F
:103A2000FCF9FAF7F9F9F801040503050AFFFB07A9
:103A300005FC070BFFF6FDF6EFFF07000104FBF5A1
:103A4000FD00FCF8030903090600FDFB030001FF6C
:103A50000001F6FCF7EEFC040608090A0B01FD0163
:103A6000F4F6FDFDFFFF00FDFE020006FC010AF773
:103A7000F701F9F6050404060606FD01FBF702FD51
:103A8000FD01FB02FBF40708FD07080405FAFCF939
:103A9000EFFB04FD0108010208000001FC0300F92E
:103AA000FE00FBF9FBFF04FF040B00FD0501FA0219
:103AB000FFF70402FCFF010300F9F90301FB03FF18
:103AC000000503010303FC0305FBF7FAFCFD03FEFD
:103AD000FD01FA0607FE0803FB0602F5FD03FC00E4
:103AE000FBFC01FCFFFEFDFD0104030600010801D3
:103AF0000005FFF5F8FBF8F9FF020101020505FEDC
:103B00000602F60708F8FD03FEF9FD01FDFB0407B8
:103B100001FDFFFFF9FF03FE03040704F5FC05FEAA
:103B2000FAFD00FBFC0404FF00FF0409020401F796
:103B3000FDFDF4F40205FD0307FDFD0301FEFE0299
:103B400006000402F700FFFA03FEFBFDF7F9FEFF93
:103B5000010302080B0B08FFFEF8F4FCFAFAF9FE69
:103B600002FF020301000406FC010601FDFAFAFC53
:103B700006060202FDFA00FFF6FBFCF3FF06000654
:103B800002060E030103FDFDFEF2F900F9FEFF033C
:103B90000604060805FFFCFFFDF4F8000004FF031F
:103BA00008020303FEFEFDFBF7F8FAFD030505001E
:103BB00001040702F9FDFA0406FA0202FD00FFFD06
:103BC0000303FBFF01FBFBF8FC0002FE04130604E9
:103BD0000901FFFCFAFAF8F5FCFEF70104FD020901
:103BE00005050A040300FC02FBFB02FDFBFFFDF2DE
:103BF000F3F9FBFF00050907060A090000010100AF
:103C0000F8F8F7FC00FAFDFDFF02FE0103FF0708CC
:103C1000FA0707FA0C0AF7FCF9F4F9F9F6F8F9FFD4
:103C2000FEFD090A05050B09060901FBFBF3F0FB84
:103C3000FEF7FD04FC0207FB0006FEFF04FE000089
:103C40001600F9EDE7FDE8DCF2FF160DF7FE28524D
:103C5000391B14F8E3DDDDD8BDB0A5C81329251A3A
:103C600018272C3F5139292705F2DFAA8D89A2D7C1
:103C7000F4FC03020D1E3B707D6C664419F5D0B256
:103C80009487909297C7E0D6E814597D7478715460
:103C90004120F5E4B685838694A6A9B9CDE9163FFF
:103CA000687A766E685221EFBF98868587868A9BF0
:103CB000AFC4E8185277797674704C17FADAA1829B
:103CC000878A87858A9AB6EB1331697E7675745D2B
:103CD00029FDDCC2A88F8784868A95AED9022A5F27
:103CE0007B78767659260DF3C7AB9C8C8585878FBC
:103CF000A8D1F323667A707272582F12FEE7CFAA0A
:103D0000888488878FADD3F610315E6E73714F3320
:103D1000290EEDDAC8A98D898B91AFD1E90A283235
:103D200042606855372A220DF3D3B19F9998A2B902
:103D3000D2E4F30A202E393A383E392209F9E8CF85
:103D4000B9AEACB3C2CEDDF402081426303234343E
:103D5000291804E9D5CFC9C0C3D0D6D6E2F4FE09EC
:103D6000161F2B352E1D120AFCEBE0D9D3D5D8D661
:103D7000DCE6E7EAFA0D181D23251F170BFDF5F405
:103D8000EFE8E6E2DBD8DCE1E9F6FF08171D1612E2
:103D90001311080301FBF5F0E8E2E2E0DCE2F0FCDD
:103DA00001060C1011100B0A0F0E0600FDF2E5E1E2
:103DB000E2E3E6EDF2F7FF0201050C100F11120E1F
:103DC0000800F8F2EDE5E2E8EFF0F0F5FAFC0005A6
:103DD00009101716110D08FEF4F0F0EFEFEDECEFFF
:103DE000F1F0F2FB04090F1414120F0902FFFBF4A7
:103DF000F1F3F3EDEAECEEF1F7FD050E12111111FE
:103E00000C030001FFFBF7F1EDEDEAE8EEF7FE022F
:103E1000080E0F0F0D0C0B0B0600FEFBF4EDEBEB89
:103E2000EAEEF3F90006090A0D0F0C0B0C0C08035F
:103E3000FBF5F1EDEAEAF0F5F8FC020507090B0DD8
:103E400010110D080501F8F1EFEFEEF0F2F6FBFEB0
:103E50000003090C0C0F12100C0700FBF7F3EFF036
:103E6000F4F5F4F7FBFE0003090E11100D0C0A0324
:103E7000FCFAF8F6F5F4F4F5F7F8F9FE0407090D85
:103E8000100E0B080401FEFBF9F9F8F6F5F6F7F849
:103E9000FC0004090C0B0A0B0A05020200FEFBF9E8
:103EA000F8F7F6F5F8FD000205080A0A0806060705
:103EB00004010000FDF9F7F8F7F8FAFE0104050522
:103EC000070807060707060401FEFCFAF8F7FAFDE3
:103ED000FDFE01030304050708080706050300FCAF
:103EE000FBFBFAFAFBFDFF00FF00030505060909CD
:103EF00007060301FFFDFCFCFDFDFCFCFDFFFF00D0
:103F00000305080807070705010000FFFDFDFDFD8B
:103F1000FDFCFCFE01020306080807060504030178
:103F2000000000FDFBFCFCFCFDFF0103050606078D
:103F30000705040404020100FFFEFCFBFBFEFFFF7B
:103F400001040505050506060504040302FFFDFD41
:103F5000FCFCFDFE0001020203050505060706053F
:103F6000030201FFFEFDFDFEFEFE0001020203044E
:103F7000060606060605030000FFFEFDFEFFFF0025
:103F80000000010304040607060504030201FFFF05
:103F900000FFFEFEFF000000000000000000000027
:103FA0000000000000000000000000000000000011
:103FB00000FF00FF0002F928686964666261605BC7
:103FC0005F533626DA939296D2DD91848E8A8F9053
:103FD000929496979B9B9DA299C4113B5674735FD4
:103FE0006E635E6F686A696763665C465562575BBD
:103FF00053261BFCE3182C303D4B4C5724EA355517
:10400000434B454741444408152DDEEF0CB88184ED
:1040100084838483838484848484848587898B8D4A
:104020008F91939597999B9C9EA0A2A4A5A7ABADB9
:10403000ABAEAFAEC7F72C27155772687D7D7A7D82
:104040007B7A78767472706E6B6968666463615FA0
:104050005D5C5A5858504F4F514925384507F7076E
:10406000031A08CAEF03D2E9E0BABAA79085908E86
:1040700081848585888A8B8F8D95ABA49E9E989D23
:104080009E9CAC9DBAF4B8B4C9E218000D140B1490
:10409000E5E03326F9495E2A2012245F3CFE405CAD
:1040A0003C5751616F394C7268696B60616660643E
:1040B000543B3034201A40252737373416362D1814
:1040C0000CEF02DCD5BCB1E3E2E0BCA9A9AAA1B522
:1040D000C9C4CAB9ADACB09193ABABA3A1ADA8BFF5
:1040E000BDB1CBA8A7E3CBC9D3EBF7D6F7FBEC1058
:1040F0001BFE09F1EA0B0629352E141B594A240927
:104100000F3245633A2E441530223950013633219F
:10411000451C2D5451603E1E4F55572B1028020050
:10412000060D060624140100D8EAFFBDCEFFE8C044
:10413000E1FBF410BF9CBEBDFF0B01F9DAE6BDD177
:10414000DFAEC8C7F505B7AAD002F2CE0AF2C4ECBA
:10415000DAFF0CDFF3DACAF0DAC3F20107F0CEEAD5
:10416000FA120FF600E0D4081908EDF9163E644281
:10417000373321444F3D341A4C3F0B4E533A3539B7
:10418000535325244B1F112A1ADACB001D18F507AB
:1041900010DDF405D3040AF604D5F1FFE6FBEFDAEF
:1041A000EA01F4F1FAEAEBD2C4E8E2CFE3E1CFCBE3
:1041B000E4E9D60C13D9E6F6D2ECF4CDF9E7DF0248
:1041C000F1031FFEEEFDCAEA06FF29FCECEDDCF868
:1041D000FBFD18240F04ECFF24201F1941350F1696
:1041E0001A2A2B3228FD03150619190D3122091838
:1041F000333D251E1513292E181A1CF10D32F90412
:1042000020ECF516FEF20304EF0205EDE8EED9EB23
:104210001EE7D8FFF5EAE5E7CCC2DEDAC2CDE6D686
:10422000D2DBDAF0E8CDDCE3EBE6D2D1CEDFE4F9A5
:104230000C030F190F191705090702F51106051CC4
:10424000FA0800121E0D1904120EFE07181F222B69
:10425000021C24FF1C19222D16151A100A222910DF
:10426000051D19F403170C001612F1FF05141706AB
:1042700002FBFAEE050B0207F50108ECD8E3E8EAC9
:10428000F7EEE8F1F1F4E5E2F9E9DBE0E3F3F4E479
:10429000E5EBF3F5E4EAEDE1FE09F8F5E9F8E1D73D
:1042A00009F8F605ECEEEEF201020102FBEFFD0E5D
:1042B000040B291C0623241824242F14142E25193A
:1042C000EDFE1E090705001D220B151D10F2F00D55
:1042D0000C0903F9FE0B11F4FE06F701F8F90BFFC8
:1042E000F4F1F5F5E8ECEAECF8FEEEF3F6E0ECF6C6
:1042F000F7F7F0E8080FDAE30103FDF0F8060D0226
:10430000F5F9FDFCF6FBFCFC0A0AFF05F8FCFCFDD8
:104310000AF20C09F30AF7E5F60F0E041204FD0D7C
:10432000FFF6F505060207FE0CFDF8071112FB0863
:10433000F3F70DF3FE0006050A15FD0702F90D0956
:1043400003F5F7131206050C13100F0C100C0D13C8
:10435000FEFAFEF90401FA05F4FD06ECFCFDFC0A88
:10436000FDEEF50FF7EC04F5F1F7EDEFF9FEF7F4DC
:10437000ECF0F7EDF4F0F4F5EAF3F1EBF4FFFFFA0B
:10438000FFFBECFB07F9FC0A08000E00F90FFE0426
:1043900010FC000D00F901060AFFFF06000A0E0DD1
:1043A000130B09101110081113070D070407FEFB6A
:1043B000020106FCF504F4F4080401FEFAF7F9061C
:1043C0000E03030B0503070501FD0200F6F3F0F4ED
:1043D000FAF9F7FEFDEFF1F3F6F5F9FFF70907F546
:1043E000FBFC04050100F90300F6FF09FDF7F5F0F9
:1043F000FBFBF000FDF300F1EBF8F90406F901FD19
:10440000F9FFFC0603FBFF090CF90608F60609FA9A
:10441000FA050B0F10090908030300080E0B0AFD2B
:10442000050CFE050D060703FD00050C02FA00FE53
:10443000FAFB00FBFBFDF60300F6FBF7FF00FCFEBA
:10444000FBFEFEF8FCF9F8FBFBFBFD00FEFBFCFCB1
:10445000FDFEF90100F7FAFD020003FFFDFCF50186
:10446000FD010BFFF7FC04FEFE09000101F9030644
:104470000204FF01070402FF0A0AFEFDFE00FAFC27
:1044800003010402FEFBF9FCFCFD0102F8FF03F747
:10449000FEFBF800FEFCF7FE03FFFDF6FD00FF0348
:1044A00002FE0103FFFF04080802040B02010406D8
:1044B000060205060908050001FFF90001FCFE00DF
:1044C000FFF9FB02F9F9040301FFF7F7FEF9FE0714
:1044D000FA0106FA0402F7FCFFFCFF06FFFD00FBF1
:1044E000FBF7FB00FCFAF4FAFDF8F7F9FCFDFFFD21
:1044F0000204FAFAFFFFFF0305020104FE0709FFA9
:1045000001FE0504FF01000300020507060001008B
:104510000602FF0701030504070103010203FC0370
:10452000FFF80300FCFCFAFFFBFDFDFCFCF900FDBD
:10453000FEFFFBFD00FFFE060600000100FD02017C
:10454000FE01FEFCFBFA00FEF7FDFEF800FF000294
:10455000FA00030205FFFCFF000101FF000100FF5C
:10456000FB00FEF6F8FBFEFDFAFAFAF7FBFCFAFF99
:1045700002FFFE04FFFD0504010405030707020313
:1045800004010405000103FF010400FC0401FE070F
:1045900000FE0600FF03030202020000FF0206FC09
:1045A000FD03FEFEFCFDFCFAFEFBFCFCFBFEFBFD3E
:1045B000FDFCFFFCF9FD01FEFEFCFDFFFEFDFD0024
:1045C000FF0303FD03FEFC01FDFCFFFF01020400ED
:1045D000FE050402020403FF0303020504000406AF
:1045E000030403FF0002FEFAFDFEFBFCFDFDFCFCE4
:1045F000FCFAFCFDFCFCFCFEFBFCFFFCFDFE00FEEF
:10460000FD02FFFF02FF0302FF02000002020101A0
:10461000010300FE010302FE00FF0002FE00000194
:1046200003000103030301020402020200FE010170
:10463000FE02040200FEFE00FFFEFF01000000017A
:10464000FF02FF00FE0101FE00FF02FF01003084B7
:1046500000000904A3093B10971C4422C1351839F6
:10466000C03F080804080403020804030202020110
:104670000108040303020202020101010101010118
:10468000010004050702882F11241FBECFEFD8E0D8
:10469000DEBFCDBF25E0A4E7B1E001C01D92A53883
:1046A000B207E1F711E0A0E0B1E0E8ECF7E702C003
:1046B00005900D92A437B107D9F713E2C4E4D3E211
:1046C00004C02197FE010E94B03AC334D107C9F754
:1046D0000E941F330C94E23B0C940000EF920F9366
:1046E000FC01628314824295407F2F70422B4383EA
:1046F000802F8295807FE82AE18200830F91EF90DE
:104700000895CF92DF92EF92FF920F931F932FB7EE
:10471000F894C0907703D0907803E0907903F090FC
:104720007A032FBF6C0D7D1D8E1D9F1D4FB7F89412
:1047300000917703109178032091790330917A03E7
:104740004FBF0C151D052E053F0528F0601771079A
:104750008207930758F71F910F91FF90EF90DF901A
:10476000CF900895AF92BF92CF92DF92EF92FF92D7
:104770000F931F93CF93DF936C017B018B01040F89
:10478000151FEB015E01AE18BF08C017D10759F025
:104790006991D601ED91FC910190F081E02DC60167
:1047A0000995892B79F7C501DF91CF911F910F9161
:1047B000FF90EF90DF90CF90BF90AF900895FC01F5
:1047C000538D448D252F30E0842F90E0821B930B76
:1047D000541710F0CF96089501970895FC01918D1C
:1047E000828D981761F0A28DAE0FBF2FB11D5D961F
:1047F0008C91928D9F5F9F73928F90E008958FEFC1
:104800009FEF0895FC01918D828D981731F0828D74
:10481000E80FF11D858D90E008958FEF9FEF0895CB
:10482000FC01918D228D892F90E0805C9F4F821B2F
:1048300091098F73992708958BE793E00E941024C4
:1048400021E0892B09F420E0822F089580E090E098
:10485000892B29F00E941C2481110C9400000895DA
:10486000FC01A48DA80FB92FB11DA35ABF4F2C91E5
:10487000848D90E001968F739927848FA689B789DC
:104880002C93A089B1898C91837080648C93938DD3
:10489000848D981306C00288F389E02D80818F7D76
:1048A00080830895EF92FF920F931F93CF93DF932E
:1048B000EC0181E0888F9B8D8C8D98131AC0E8895C
:1048C000F989808185FF15C09FB7F894EE89FF892B
:1048D0006083E889F98980818370806480839FBFC9
:1048E00081E090E0DF91CF911F910F91FF90EF90C9
:1048F0000895F62E0B8D10E00F5F1F4F0F731127D9
:10490000E02E8C8D8E110CC00FB607FCFACFE88913
:10491000F989808185FFF5CFCE010E943024F1CF47
:10492000EB8DEC0FFD2FF11DE35AFF4FF0829FB787
:10493000F8940B8FEA89FB8980818062CFCFCF9377
:10494000DF93EC01888D8823B9F0AA89BB89E889B7
:10495000F9898C9185FD03C0808186FD0DC00FB65D
:1049600007FCF7CF8C9185FFF2CF808185FFEDCFDB
:10497000CE010E943024E9CFDF91CF9108953FB757
:10498000F89480919D0290919E02A0919F02B09117
:10499000A00226B5A89B05C02F3F19F00196A11DC6
:1049A000B11D3FBFBA2FA92F982F8827BC01CD0179
:1049B000620F711D811D911D42E0660F771F881FD8
:1049C000991F4A95D1F70895FC01818581111186BF
:1049D0002381348145815681D901A41BB50B42172F
:1049E000530718F0DA01A21BB30B9781992309F141
:1049F0007081519780F0711110C061E06083128264
:104A0000118260816623E9F024173507D1F03683DF
:104A10002583892F08957723A1F0A181B2816A0FA0
:104A20007B2F711D72836183603D774068F3108234
:104A3000E8CFAB2B29F081E080833683258308956E
:104A4000108208950F931F93DC01ED91FC91119753
:104A500001E010E020E030E004C0000F111F221F31
:104A6000331F6A95D2F7442339F00E2B1F2B0D9379
:104A70001C931F910F910895009510950E231F23ED
:104A8000F6CFEF920F93CF93DF93A62FB0E0EC0118
:104A9000EB81FC81EA0FFB1F4083AD01440F551FE2
:104AA000EF81F885E40FF51F11821082ED81FE8100
:104AB000EA0FFB1F30813F7040E1249FE001112489
:104AC0002C2F232B2083EC01ED81FE81EA0FFB1FAD
:104AD0002081207F0F70022B00834E2DDF91CF911C
:104AE0000F91EF900C9422252A9870E062FB8827A2
:104AF00080F986608EBD0DB407FEFDCF8EB586E0D1
:104B0000660F771F8A95E1F76EBD0DB407FEFDCFE6
:104B10008EB51EBC0DB407FEFDCF9EB52A9A8F70D0
:104B20008927982789270895CF92DF92FF920F93C4
:104B30001F93CF93DF93DC01A657BF4FC1E9D1E0AC
:104B400040E0BC0162557F4F6C0123EBC20ED11CCB
:104B500051E012E103E085EEF82E2D913C91119782
:104B6000411116C0FB018081982F9D7F913009F47F
:104B700034608250823008F43860F6018081982FCA
:104B80009D7F913009F431608250823008F43260A8
:104B9000899199918217930741F1CE010297FC0107
:104BA00031832083952F941B809176038111FCCF54
:104BB000809175038111F8CF8091BC0084FDF4CF02
:104BC0001093F3022093F4023093F5020093F20263
:104BD000509376031092F1028091F1029062990F46
:104BE000982B9093F102F092BC005296413041F420
:104BF000DF91CF911F910F91FF90DF90CF9008959B
:104C000041E0ABCFCF93DF93FC0140815181862FF0
:104C100090E02381222369F0C681C40FD52FD11DD6
:104C20006881278130E0860F911D2817390708F425
:104C3000C901A581A40FB52FB11D4481489F9001E2
:104C4000499F300D11243C9326812F5F26833281AA
:104C5000231710F0231B268326814381240F23175B
:104C600020F42583DF91CF910895231BFACF0F9372
:104C70001F93CF93DF93E42FF0E0F595E795A62FF0
:104C8000B0E0342F3170C32F30E0D32FAA0FBB1FF9
:104C9000A80FB91FAE0FBF1F50963C915097E22F3F
:104CA0008E01000F111F000F111F01C0EE0F0A959A
:104CB000EAF7E327CD5EDE4F5881E523E3275096E0
:104CC000EC93DC0190968D919C91009759F0DC015A
:104CD000ED91FC910280F381E02DDF91CF911F9146
:104CE0000F910994DF91CF911F910F910895342F67
:104CF000DC0114964C91149746130CC018968D91B4
:104D00009C91DC01ED91FC910680F781E02D422F12
:104D1000632F099408950F931F93CF93DF932F7000
:104D2000413051F0F0F0423009F1433039F1DF9178
:104D3000CF911F910F91089570E0675F7F4F660FCD
:104D4000771FFC01E60FF71F0190F081E02D238310
:104D50008681280F25838281281748F3281B258305
:104D6000E6CFFC01E60FF11D22A3E1CFE62FF0E034
:104D700026952F5FEF55FD4F2083D9CF70E0DB01E3
:104D8000A757BE4F1C92660F771FFB01E05BF94BE4
:104D900005911491FB01EE5AF94B45915491415004
:104DA0005109EB01C758DE4F2F3081F459834883F6
:104DB000FB01E758FE4F80819181880F991F880F72
:104DC000991F9183808381E08C93B1CF211103C01F
:104DD00019830883EDCFCA01801B910B019634E043
:104DE000969587953A95E1F7289FF001299FF00D58
:104DF0001124E00FF11F9F012F5F3F4F598348831C
:104E0000E258F94F84914217530790F2F901E258A2
:104E1000F94FE49187FF08C0E7FD06C0FB01E758A2
:104E2000FE4F31832083C4CF2F5F3F4F8E2FEBCFB8
:104E3000CF92DF92EF92FF92CF93DF93EC01E62FB8
:104E4000F0E07796EE0FFF1FE80FF91F51834083C4
:104E50008EA59FA528A939A9820F931FCAA4DBA4F8
:104E6000ECA4FDA482332DE09207F0F40097F1F456
:104E700081E1C8168BE2D806E104F10471F081E10A
:104E80009BE2A0E0B0E08AA79BA7ACA7BDA78BEAF6
:104E900095E09093890080938800DF91CF91FF90F7
:104EA000EF90DF90CF90089581E39DE060E073E0A4
:104EB0000E947D3AFB01EE0FFF1FE859F94F259143
:104EC0003491FC01EE0FFF1FE859FF4FA591B491FB
:104ED0000E946E3A59E096958795779567955A9511
:104EE000D1F7E4E0660F771FEA95E1F79B0150E008
:104EF00040E02C153D054E055F0579F22AA73BA73A
:104F00004CA75DA760E074E284EF90E00E944C3A09
:104F10003093890020938800C0CF089561110FC09D
:104F2000DC011696ED91FC91448380859185DC012E
:104F3000ED91FC910190F081E02D642F0994613096
:104F400071F4DC011696ED91FC9145838085918585
:104F5000DC01ED91FC910280F381E02DEECF08950C
:104F6000EF920F93DC0118964C91B5E06B9FF00126
:104F70001124E255FF4FDC0114968D919C91EE2493
:104F8000E39402E0242F68E08E0F9F1F0E946E239F
:104F90000F91EF9008950F931F93CF93DF93FC0130
:104FA0006430D9F44E5D5F4F2FE0249FC001259FF0
:104FB000900D1124AC01452F55274695469536E0B6
:104FC000440F551F3A95E1F760E086819781DF91A4
:104FD000CF911F910F910C9418276230A1F42FEFFD
:104FE0003FE0241B350BA1E3BDE00E946E3AAB010C
:104FF000BC019CE076956795579547959A95D1F7B2
:10500000407E61E0E2CF61111DC04E5D5F4F8FE0D9
:10501000849F9001859F300D1124232F33272695DF
:105020002695838990E02817390708F4C901228D55
:105030002817190611F0828F138EDF91CF911F91DF
:105040000F910895DC01A60FB11D1A968C91843042
:10505000A0F78F01080F111DD8015C969C91951740
:1050600061F3EA010680F781E02D2D2F482F64813E
:10507000828193810E943726F801D48FDECFDC0134
:1050800012968D919C91DC01ED91FC910280F3814F
:10509000E02D09940895DC0112968D919C91DC011C
:1050A000ED91FC910190F081E02D09947F928F9217
:1050B0009F92AF92BF92CF92DF92EF92FF920F93A7
:1050C0001F93CF93DF93CDB7DEB7A0970FB6F894B9
:1050D000DEBF0FBECDBF8C01762E862F90E08058AC
:1050E0009F4F65E0880F991F6A95E1F7209176033D
:1050F0002111FCCF209175032111F8CF2091BC0024
:1051000024FDF4CF9093F3028093F40282E0809325
:10511000F20281E0809376031092F1028091F10215
:10512000806A8093F10285EE8093BC0080917603C3
:105130008111FCCF8091BC0084FDF8CF80E2809388
:10514000F20281E0809375038093F1028091F10275
:10515000806A8093F10285EE8093BC008091750394
:105160008111FCCF8091BC00982F9071E92E84FDB5
:10517000F5CF80E2E3EFF2E0DE01119601900D92AF
:105180008A95E1F7FE0131966F0158019E012F5E6D
:105190003F4FD80188248394408181814F3F11F48F
:1051A0008F3F09F0812C90E0982F8827840F911D64
:1051B0008D939D933296E217F30771F7912CF601C8
:1051C000F088FFEFFF12812C2F2D2F7040E0692D0A
:1051D000C8010E9437262F2D207F30E094E03595BE
:1051E00027959A95E1F741E0692DC8010E9437267D
:1051F000F601F188FFEFFF12812C2F2D2F7042E076
:10520000692DC8010E9437262F2D207F30E084E0D1
:10521000359527958A95E1F743E0692DC8010E94ED
:105220003726939482E0C80ED11C98E09912C7CF1C
:10523000882001F1F501119211925F012FE040E009
:105240006E2DC8010E94372620E041E06E2DC80176
:105250000E94372627E042E06E2DC8010E943726C3
:105260002FE043E06E2DC8010E943726E394F8E05A
:10527000EF12E0CFF80172A2A0960FB6F894DEBF4D
:105280000FBECDBFDF91CF911F910F91FF90EF9097
:10529000DF90CF90BF90AF909F908F907F900895B8
:1052A0001F93CF93DF93EC01162F6E83888599852A
:1052B000DC01ED91FC910480F581E02D099511113F
:1052C00016C06F816F3F99F08AA9882381F08A8187
:1052D0009B810E94562888859985DC01ED91FC917F
:1052E0000084F185E02D6F8109958FEF8F83DF9129
:1052F000CF911F91089580917105909172059093BF
:105300007405809373058091630590916405FC0199
:1053100012AA60E00E945029E0916305F0916405B3
:1053200082A9882311F08FEF878380916105909186
:1053300062050C949425AF92BF92CF92DF92EF92C8
:10534000FF920F931F93CF93DF93442309F461C01F
:10535000EC01EE81FF8182A9882309F465C0668192
:105360006F5F6F70CF010E945029888D998D880FD3
:10537000991F9F8B8E8B198E188EEE80FF805701A0
:1053800082E1A80EB11C6701D0E0C0E0D5018D918B
:105390009D915D01D7011296ED91FC9113978E01BD
:1053A000000F111FE00FF11F16964C9120813181E3
:1053B00002C0369527954A95E2F760E020FF02C0CB
:1053C000F60162A10E9402268823D9F090E0FC0138
:1053D000EE58F94BE491DE01AF51BD4FEC938E597D
:1053E000994BFC018491FE01E752FD4F8083F80147
:1053F000E753FD4F80819181F801E754FD4F918380
:1054000080832196FFEFCF1ADF0AC830D10509F05B
:10541000BDCFDF91CF911F910F91FF90EF90DF9063
:10542000CF90BF90AF90089581E082ABA4CFEF9270
:105430000F931F93CF93DF93EC01162F49858C8137
:105440009D8122E0E22E01E0242F6FEF82559F4FD5
:105450000E946E230E80DF81C02D8AA9811119C0A0
:105460001F3F89F0612F8A819B810E945628888581
:105470009985DC01ED91FC910084F185E02D612F8F
:1054800009958FEF8F83DF91CF911F910F91EF904F
:1054900008951F83F8CFCF92DF92EF92FF920F9380
:1054A0001F93CF93DF93EC01AE81BF811596FC90E3
:1054B0001597EC81FD8114962C91C22ED12CE657C4
:1054C000FF4F81E090E002C0880F991F2A95E2F714
:1054D000918380830C811D8104561F4FF801428106
:1054E00050E070E060E0838194810E94DB3BF80132
:1054F00011821082EC81FD81AE81BF8112960D90E8
:10550000BC91A02DC601880F991FA80FB91F2D911E
:105510003C91E456FF4F31832083EE81FF8122814D
:105520003381820F931FFC01208131810F2C02C037
:10553000369527950A94E2F78C819D818D549F4F73
:1055400020FF18C022E0FC0120838C819D81EE2485
:10555000E394088529854FEF6F2D84569F4F0E9455
:105560004125DF91CF911F910F91FF90EF90DF9038
:10557000CF90089521E0FC0120838C819D81E12C56
:1055800009852885E8CF6F927F929F92AF92BF9254
:10559000CF92DF92EF92FF920F931F93CF93DF93FF
:1055A000CDB7DEB7A0970FB6F894DEBF0FBECDBF64
:1055B0008C01862FF801A681B78114966C911497FF
:1055C0008111B2C00480F581E02D413021F4E25513
:1055D000FF4F82E090C0DF01AA57BF4F0D90BC91F2
:1055E000A02D1A968D919C91813D974008F498C00A
:1055F000E255FF4F128281818F708083D80114960B
:10560000ED91FC911597E255FF4F81E0808316964E
:10561000ED91FC9142815381262F30E020583F4F7D
:1056200095E0220F331F9A95E1F77A01FE0131963A
:105630005A01B0E1AB0EB11C6F013A01CF01D301A9
:105640009C9011967C91B2E06B0E711CD6019C92DD
:1056500011967C93B2E0CB0ED11C6A147B0479F7CF
:105660006F0170E1C70ED11CD70150967C91509705
:10567000708B51967C91718BB2E0EB0EF11C3296DF
:10568000EC15FD0589F7709176037111FCCF7091CF
:1056900075037111F8CF7091BC0074FDF4CF309395
:1056A000F3022093F40220E2FC01A5EFB2E00190A6
:1056B0000D922A95E1F722E22093F20221E0209355
:1056C00076031092F1022091F102206A2093F102F8
:1056D00025EE2093BC00FA0162A3698341E050E00B
:1056E00064EF73E00E942A3AD8011496ED91FC9180
:1056F000E255FF4F81E08083A0960FB6F894DEBF9D
:105700000FBECDBFDF91CF911F910F91FF90EF9012
:10571000DF90CF90BF90AF909F907F906F90089553
:10572000C8010E94172AE0CF813031F7E480F5806C
:10573000413021F4F701ED54FF4F4BCFC70188579B
:105740009F4FFC0180819181FC0182859385813D81
:10575000974040F1F701ED54FF4F128281818F7025
:105760008083D8011496ED91FC911597EA57FF4F6D
:105770000190F081E02D248116968D919C9122FF5D
:1057800007C060E00E945029C8010E944B2AB4CF94
:10579000DC011296ED91FC9180E1DF011D928A956A
:1057A000E9F7F2CF15964C91159712960D911C9131
:1057B000E62FF0E0EE0FFF1FE00FF11FE080F18019
:1057C0006701042E02C0D694C7940A94E2F79601AA
:1057D0002095309581E090E0A0E0B0E0042E04C078
:1057E000880F991FAA1FBB1F0A94D2F7C0FC13C0D1
:1057F0008E299F2991838083F80180A191A1009730
:1058000009F47ACF2170DC01ED91FC910190F081D7
:10581000E02D099571CF809590958E219F21EACF3B
:105820001F920F920FB60F9211242F933F934F9315
:105830005F936F937F938F939F93AF93BF93EF93F8
:10584000FF938BE793E00E943024FF91EF91BF918B
:10585000AF919F918F917F916F915F914F913F9108
:105860002F910F900FBE0F901F9018951F920F92BF
:105870000FB60F9211242F938F939F93EF93FF9363
:10588000E0918B03F0918C038081E0919103F09182
:10589000920382FD1BC09081809194038F5F8F7370
:1058A00020919503821741F0E0919403F0E0E558D0
:1058B000FC4F958F80939403FF91EF919F918F916F
:1058C0002F910F900FBE0F901F9018958081F4CFED
:1058D0001F920F920FB60F9211242F933F938F9325
:1058E0009F93AF93BF938091770390917803A0919A
:1058F0007903B0917A0330919C0223E0230F2D3776
:1059000058F50196A11DB11D20939C028093770349
:1059100090937803A0937903B0937A0380919D02CA
:1059200090919E02A0919F02B091A0020196A11DAC
:10593000B11D80939D0290939E02A0939F02B0930D
:10594000A002BF91AF919F918F913F912F910F90A6
:105950000FBE0F901F90189526E8230F0296A11DE9
:10596000B11DD2CF1F920F920FB60F9211248F93B9
:105970009F93EF93FF938091B900887F8832D9F18C
:10598000D0F4803171F168F4882379F0883049F1DE
:10599000FF91EF919F918F910F900FBE0F901F90ED
:1059A0001895883141F1803299F784E98093BC00E1
:1059B00010927603EDCF803409F441C030F4803387
:1059C000A1F3883329F785E9F1CF803559F188357E
:1059D000F1F18834E9F684E98093BC0010927503F4
:1059E000D7CF8091F1028093BB0085EC8093BC00FF
:1059F00010929B02CDCF90919B028091F20298175A
:105A0000A0F6E0919B02F0E0ED50FD4F8081809385
:105A1000BB0080919B028F5F80939B0285EC8093FB
:105A2000BC00B6CFE0919B02F0E08091BB00ED504E
:105A3000FD4F808380919B028F5F80939B029091AA
:105A40009B028091F202981748F385E8E8CFE09135
:105A50009B02F0E08091BB00ED50FD4F8083BBCFF7
:105A60001F920F920FB60F9211242F933F934F93D3
:105A70005F938F939F93EF93FF9389B18095EEE4AB
:105A8000F6E49491982320919902921709F43CC06E
:105A9000282F30E0E2E8F6E45491E3E8F6E444919C
:105AA000F90102C0F595E7955A95E2F7EE0FFF1F51
:105AB000EE0FFF1FE470FF2702C0359527954A952A
:105AC000E2F7F3E0220F331FFA95E1F7287033274E
:105AD0002E2BE0919702E695E695E22BE093970254
:105AE0000E2E000CFF0BE25CF94BE4912091E902D1
:105AF0003091EA022E1B3109E7FD33953093EA021B
:105B00002093E90290939902EFE4F6E4249128238C
:105B100090919A02921709F43BC090E0E4E8F6E411
:105B20004491E5E8F6E43491FC0102C0F595E7956F
:105B30004A95E2F7EE0FFF1FEE0FFF1FE470FF27FD
:105B400002C0959587953A95E2F753E0880F991F23
:105B50005A95E1F7887099278E2BE0919802E69587
:105B6000E695E82BE09398020E2E000CFF0BE25C0A
:105B7000F94BE4918091EB029091EC028E1B91091C
:105B8000E7FD93959093EC028093EB0220939A02A9
:105B9000FF91EF919F918F915F914F913F912F9145
:105BA0000F900FBE0F901F9018951F920F920FB677
:105BB0000F9211248F939F93EF93FF9383B180955E
:105BC000982F9170EEE5F4E0908386958170818343
:105BD000FF91EF919F918F910F900FBE0F901F90AB
:105BE00018951F920F920FB60F9211248F939F93C7
:105BF000EF93FF938091790090919602913059F044
:105C00009230B9F1FF91EF919F918F910F900FBE5C
:105C10000F901F901895E0919502F0E08058EB5698
:105C2000FE4F8083E0919502F0E0EB56FE4F8081BD
:105C300087FD16C0E0919502E150FF0BEB56FE4F39
:105C4000808187FF0DC082E080939602E0919502EB
:105C5000F0E0EB56FE4F8081809395011092950203
:105C6000809195028F5F809395028EEC80937A00ED
:105C7000C9CFE0919502F0E08058EB56FE4F80834B
:105C8000809195028F3F21F483E080939602BACFF2
:105C9000E0919502F0E0EB56FE4F808187FDE0CF6A
:105CA000E0919502E150FF0BEB56FE4F808187FF9C
:105CB000D7CF9091950280910201981788F284E0E5
:105CC000E4CF78941F920F920FB60F9211242F9366
:105CD0003F934F935F936F937F938F939F93AF9374
:105CE000BF93CF93DF93EF93FF9390E080E050E07A
:105CF00040E0FC01E757FE4F60819C01220F331FFB
:105D00006623D1F0D901A754BD4F0D90BC91A02DB1
:105D1000E901C753DD4F68817981A617B70761F4A0
:105D2000D901A758BE4F6D917C91D901A755BD4FA0
:105D300011967C936E931082D901A754BD4F6D913B
:105D40007C91119727553D4FF9012081318126170C
:105D5000370788F1ED91FC911197F695E795F69547
:105D6000E795E258F94FE4910E2E000CFF0BEC0181
:105D7000CF51DD4F2881BF0102C0759567952A95E7
:105D8000E2F7460F571FEC01C752DD4F288102C0D2
:105D9000F595E7952A95E2F74E0F5F1FFC01EF5549
:105DA000FD4F20816D917C911197260F372F311D6A
:105DB00011963C932E9301968830910509F099CF66
:105DC00040385105B4F08FEF8093B400FF91EF910C
:105DD000DF91CF91BF91AF919F918F917F916F9103
:105DE0005F914F913F912F910F900FBE0F901F9099
:105DF000189540387FEF57071CF41092B400E6CF97
:105E000040584093B400E2CF909176039111FCCFBB
:105E1000909175039111F8CF9091BC0094FDF4CF4F
:105E20006093F3021092F40292E09093F20291E0F8
:105E3000909376031092F1029091F1028062880FA4
:105E4000892B8093F10285EE8093BC000895CF9258
:105E5000DF92EF92FF920F931F93CF93DF9300D0C7
:105E6000CDB7DEB77C011A8219828B01085F13401F
:105E70006801D694C794D694C79442E050E0CE010E
:105E800001960E941A3AC601880F991F880F991F20
:105E9000F801E81BF90BF695E7958601000F111F35
:105EA0000C0D1D1DE00FF12FF11DFD96EE0FFF1FD4
:105EB000EE0DFF1D898190E0982F88272A81820F9F
:105EC000911D9183808326E02C9DC0012D9D900D16
:105ED0001124E80EF91EF701E258FF4FD701A4582C
:105EE000BF4F8AE7E80EF11C8D919C91D7012D914F
:105EF0003C91821B930B918380830F900F90DF91D5
:105F0000CF911F910F91FF90EF90DF90CF90089568
:105F10008F929F92AF92BF92CF92DF92EF92FF92B9
:105F20000F931F93CF93DF9310927E0310927D0304
:105F300088EE93E0A0E0B0E080937F03909380032D
:105F4000A0938103B093820389E191E090937C0355
:105F500080937B0385EC90E0909388038093870384
:105F600084EC90E090938A038093890380EC90E026
:105F700090938C0380938B0381EC90E090938E033D
:105F800080938D0382EC90E09093900380938F0335
:105F900086EC90E090939203809391031092940387
:105FA00010929503109296031092970310921E047C
:105FB00010921F04109220041092210410922204C7
:105FC00010922304109224041092250410922604A7
:105FD00010922704109228041092290410922A0487
:105FE00010922B0410922C0410922D048FE391E058
:105FF00090935E0580935D0589E591E0909360053F
:1060000080935F05809155058111CCC083E391E0B9
:1060100090939C0480939B0410929F041092A1047F
:106020001092A0041092A3041092A20481E0809325
:10603000A40490E19093A5048093A6041092A70471
:106040001092A8041092A9041092AA041092AC0411
:106050001092AB041092AE041092AD048093AF0482
:106060009093B0048093B1041092B2041092B304E0
:106070001092B404E5EBF4E088E0DF011D928A950C
:10608000E9F7EDEBF4E091E08FEF108212821182DC
:1060900014821382168215829783808711863A961E
:1060A000B5E0ED30FB0789F788E0DF011D928A95A6
:1060B000E9F7E5E1F5E08CE0DF011D928A95E9F76B
:1060C000C5E2D5E010E1198218821C861B861E8667
:1060D0001D861F86198A188A80E190E00E94B63AD0
:1060E0009C01205F3F4FFC011192E217F307E1F79B
:1060F0009C838B8380E190E00E94B63A9C01205FF4
:106100003F4FFC011192E217F307E1F79E838D8365
:1061100080E290E00E94B63A9C01205E3F4FFC0175
:1061200011921192E217F307D9F798878F8380E1D4
:1061300090E00E94B63A9C01205F3F4FFC01119213
:10614000E217F307E1F79A8789871A8380E09A813B
:10615000891738F4E985FA85E80FF11D80838F5F90
:10616000F6CF6296B5E0C934DB0709F0ACCF1092E8
:10617000490510924A0510924B0510924C05109259
:106180004D0510924E0510924F0510925005109239
:10619000510510925205109253051092540581E05A
:1061A000809355058BE994E0909362058093610597
:1061B00080919304811132C08BE291E0909361044D
:1061C0008093600410926404109265041092660437
:1061D0008FEF8093670488E0EAE6F4E0DF01282F80
:1061E0001D922A95E9F7E2E8F4E0DF011D928A9515
:1061F000E9F710928A0410928B0410928C0410928A
:106200008D0410928E0410928F04109290041092BC
:1062100091041092920481E080939304C0E6D4E04C
:10622000D0936405C093630584E08093650588E09E
:1062300080936605EBE0F1E0A7E6B5E0982F0190CA
:106240000D929A95E1F793E090936F0595E1909305
:10625000700520ED37E0309372052093710530937F
:1062600074052093730510927605109275051092AF
:10627000770510927805E9E7F5E0DF011D928A9530
:10628000E9F78FE595E0909369048093680483E2D1
:1062900090E00E94B63AFC0180E1DF01282F1D92B8
:1062A0002A95E9F79F01205F3F4FD9011D928A95FA
:1062B000E9F78FEF82A3D1A3C0A3F0936304E09327
:1062C00062048DE595E090939E0480939D04F8947C
:1062D0002A9A229A8CB580618CBD8CB580648CBD65
:1062E000239A259A8DB581608DBD8CB58D7F8CBD2F
:1062F0008CB581608CBD8CB58F7D8CBD8CB5877F56
:106300008CBD8CB58B7F8CBD68EF73E08BE994E01E
:106310000E94272F6AEF73E08BE994E00E94272FF9
:106320006CEF73E08BE994E00E94272F6EEF73E02F
:106330008BE994E00E94272F55EBE52E54E0F52ED3
:10634000CBE9D4E010E001E099249A9466E0862E2F
:10635000CC24CA947FE0D72E5701F70180818111A8
:106360003AC0812F8B7F612F09F058C18BE994E0EF
:106370000E94742541E050E0143011F450E040E0F8
:10638000B0E0A0E0849E9001859E300D112425563A
:106390003B4FF901E658FF4F40815181BC01CD01CF
:1063A000641B750B810991094BE0660F771F881FED
:1063B000991F4A95D1F722583F4FD9012D913C9111
:1063C00050E040E00E94913ADA01C9019C5FAF4F72
:1063D000BF4FB7FF08C01AA21CA21BA21EA21DA27B
:1063E00018A61FA20EC01AA21CA21BA28115E0E1D2
:1063F0009E07A105B1050CF418C1DEA2CDA2D8A656
:10640000CFA209A79AA61BA6FFEFEF1AFF0AD50194
:106410008C91F701E95AFF4F5F01813009F00AC101
:10642000612F8BE994E00E94742521E0813098402F
:1064300008F420E0D5012C931F5F2A96183009F04C
:106440008BCF1092EC041092C40410927C008091C7
:106450007C00806480937C0080917C0080628093CB
:106460007C0090E080E0812C912C5401839430E0FA
:1064700020E0BC016E57794BFB01E20FF31F449102
:106480005AB17501640104C0CC0CDD1CEE1CFF1C6C
:106490004A95D2F7C094D094E094F094452F4C21C3
:1064A0004AB9E4914BB17501640104C0CC0CDD1C08
:1064B000EE1CFF1CEA95D2F74C294BB9213031056F
:1064C00009F0BAC002968430910589F62098289880
:1064D0002198299856985E98539A5B98C3B1C095B5
:1064E0008C2F817080935E048CE090E00E94B63A1D
:1064F000FC0113821782168211861086138612867B
:106500008BE9E82E84E0F82EF182E082128212E01C
:106510001583D1E0D483F0932205E0932105C6953D
:10652000C170C0935F048CE090E00E94B63AFC0119
:106530001382178216821186108613861286F182C4
:10654000E082D2831583D48390932405809323051E
:1065500080916B00816080936B0080916B00826002
:1065600080936B00D89A8091680081608093680066
:1065700080916D00846080936D0080916D008061DA
:1065800080936D0080916D00806280936D0080919A
:106590006D00806480936D0080916D0080688093B1
:1065A0006D00DA9A8091680084608093680088E0CA
:1065B0008093A50480919F0488301CF087E080932D
:1065C0009F0478948091B9008E7F8093B900809168
:1065D000B9008D7F8093B90088E48093B80085E48A
:1065E0008093BC0060E080E00E94042F61E080E0C6
:1065F0000E94042F60E081E00E94042F61E081E0AE
:10660000DF91CF911F910F91FF90EF90DF90CF908E
:10661000BF90AF909F908F900C94042F8BE994E0E3
:106620000E9474251AA21CA21BA29EA38DA398A748
:106630008FA3E7CE108200CF21E030E01DCFCF93B3
:10664000DF9300D01F92CDB7DEB7789484B5826017
:1066500084BD84B5816084BD85B5826085BD85B506
:10666000816085BD80916E00816080936E00109284
:1066700081008091810082608093810080918100FF
:106680008160809381008091800081608093800090
:106690008091B10084608093B1008091B0008160EE
:1066A0008093B00080917A00846080937A0080911A
:1066B0007A00826080937A0080917A008160809372
:1066C0007A0080917A00806880937A001092C100ED
:1066D00010925A0410925B0410925C0410925D04B4
:1066E00010921A0410921B0410921C0410921D04A4
:1066F00068EB7BE080E090E00E9481230E94BF2451
:106700004B015C0198EEC92E93E0D92EE12CF12CBF
:106710000E94BF24681979098A099B09683E734061
:1067200081059105A8F321E0C21AD108E108F1081A
:1067300038EE830E33E0931EA11CB11CC114D104AA
:10674000E104F10429F7E0918B03F0918C0382E0DE
:106750008083E0918703F09188031082E0918903A0
:10676000F0918A0380E1808310929303E0918F037C
:10677000F091900386E08083E0918D03F0918E0389
:10678000808180618083E0918D03F0918E03808110
:1067900088608083E0918D03F0918E038081806812
:1067A0008083E0918D03F0918E0380818F7D8083C3
:1067B0002FB7F8948091770390917803A091790393
:1067C000B0917A032FBF80931A0490931B04A09377
:1067D0001C04B0931D0440E150E063E671E08BE7D8
:1067E00093E00E94B2236AE070E080E090E00E94B3
:1067F000812381E080932E04E0916105F091620590
:106800008387868B81A30091630510916405809135
:10681000B6008F7B8093B6008091B6008F7D809309
:10682000B6008091B00081608093B0008091B0008C
:1068300082608093B0008091B100877F8093B10027
:106840008091B0008F7E8093B0008091B000806214
:106850008093B0008091B0008F7B8093B0008091D6
:10686000B0008F778093B0008091B10081608093F9
:10687000B1008091B1008D7F8093B1008091B10013
:106880008B7F8093B100F894809180008E7F8093FD
:106890008000809180008D7F8093800080918100B6
:1068A000886080938100809181008F7E8093810039
:1068B00080918100816080938100809181008D7F33
:1068C00080938100809181008B7F809381008091F3
:1068D0000301909104019093890080938800809136
:1068E0006F00826080936F007894F80182A593A571
:1068F000A4A5B5A581319B42A105B10579F081E13F
:106900009BE2A0E0B0E0F80182A793A7A4A7B5A7F7
:106910008BEA95E090938900809388005801F2E11A
:10692000AF0EB11C780122E2E20EF11CA0E17A2E3A
:10693000BFE08B2E80E8982E88E090E00E94B63A67
:106940006C01DC0113961C92139715961C921597F7
:1069500016961C92169712967C9280E190E00E9407
:10696000B63AF60191838083D501CD92DD925D0127
:1069700087829482EA16FB06F9F640E556E489EC34
:10698000C82E82E0D82E61EE72E0A9EDB2E0570188
:1069900090E080E021E8822E26E4922E31E7632EFB
:1069A00036E4732EE4E05E2EFFE04F2EFA012591CF
:1069B0003491F6013183208332966F019C01220FBE
:1069C000331FF901E753FD4F20803180220C331C27
:1069D000220C331C318220824E5F5F4FFA01E5901A
:1069E000F490F1E0EF1AF108F901E755FD4FF1825B
:1069F000E082E080F180EE0CFF1CEE0CFF1CF182C7
:106A0000E082E080F18027543D4FF901F182E0827D
:106A1000F4012491FB012193BF01F30124912D93F3
:106A2000FC01EF55FD4F5082F50141925F01019647
:106A30008830910509F0BACFD80114961C921497AA
:106A400018968D919C91DC01ED91FC910190F08163
:106A5000E02D60E00995F801158280859185DC01C3
:106A6000ED91FC910280F381E02D60E0099560E0FA
:106A7000C8010E945029E0916305F09164050281EC
:106A8000138141E050E064EF73E0CE0101960E9473
:106A90001A3A69816770C8010E9456288DE595E011
:106AA0000E944B2A40916505809161059091620595
:106AB000F2E0EF2E01E0242F64E082559F4F0E9408
:106AC0006E23662463948FB7F894409177035091B6
:106AD00078036091790370917A038FBF8091ED0202
:106AE0009091EE02A091EF02B091F002F42EF81A0C
:106AF0008F0D911DA11DB11D8093ED029093EE02AB
:106B0000A093EF02B093F00200916105109162052D
:106B10001801BAE12B0E311C6801E12CF801E75491
:106B2000FF4FFB83EA832801FAE44F0E511CD10189
:106B30008D911D01772473947E0CF6013A965F01C6
:106B40008111AFC04601F2E28F0E911C8E2D8B7F1A
:106B50006E2D09F07DC0C8010E94742541E050E00F
:106B600024E0E21202C050E040E0B0E0A0E066E0C5
:106B7000649F9001659F300D1124200F311FF90192
:106B8000E658FF4F40815181BC01CD01641B750B5C
:106B900081099109EBE0660F771F881F991FEA951D
:106BA000D1F722583F4FD9012D913C9150E040E060
:106BB0000E94913ADA01C9019C5FAF4FBF4FB7FF06
:106BC00035C0F60116A215A260E0C4010E94E424BB
:106BD000882309F466C0D80112968D919C91DC013E
:106BE000ED91FC910480F581E02DD6019A962C91CF
:106BF0009A9795964D915C912F3FA9F034E0569568
:106C000047953A95E1F730E02F5F3F4F429FB00143
:106C1000439F700D529F700D1124AB0164E0569597
:106C200047956A95E1F76E2D09953BC08115F0E116
:106C30009F07A105B10544F0EFEFFFE0D60196965E
:106C4000FC93EE939597C0CFF60196A385A3BCCF96
:106C5000C8010E947425F60196A385A36F2DC40177
:106C60000E94E4248823E9F0D60195964D915C9129
:106C7000B5E0EB1211C1EA81FB81808180FF26C162
:106C800094E0569547959A95E1F7D20118968C9124
:106C90001897841709F434C319966C9219971896AB
:106CA0004C93E72C6501B8E07B1241CFC0906105A1
:106CB000D09062058601065E1F4FE12CF80181919C
:106CC0008F018130E1F46E2DC6010E94742541E0F0
:106CD0008130984008F440E0F801E95AFF4F808184
:106CE000481769F04083D60112968D919C91DC0182
:106CF000ED91FC910284F385E02D6E2D0995E394CE
:106D0000B8E0EB12DBCFC0906105D0906205E6E8F9
:106D1000CE0ED11CB12CA12C8F2C912CD6010D9113
:106D20001D916D01F501E25AFB4F8081E62CE81AB6
:106D3000F801848181FFD8C0268137812F3F320737
:106D400039F0280D391DD80117963C932E931697CC
:106D5000F801268137812431310508F4CDC08D7FBB
:106D60008483F8018581823009F4A2C180859185F0
:106D70008F3F980739F0880D991DD80119969C937B
:106D80008E931897F801848187FF18C080859185BC
:106D9000883C910598F0838181110CC0808191819C
:106DA000DC01ED91FC910280F381E02DD801129677
:106DB0006C910995F80184818F778483D8011496AA
:106DC0008C91149783FF0AC018962D913C911997C6
:106DD000283C310518F0877F14968C93F801828542
:106DE00093858F3F980739F0880D991DD8011B9620
:106DF0009C938E931A97F8018481982F9170E916CD
:106E0000F9F082FF1DC085FD1BC022853385203D22
:106E10003740B0F08062D80114968C931497139683
:106E20008C91139781110CC08D919C91DC01ED9197
:106E3000FC910680F781E02DD80112966C9109959E
:106E4000F8018581E81609F457C0E5828481982FFE
:106E50009170E916D1F01386128684608483838151
:106E600081110DC080819181DC01ED91FC91019037
:106E7000F081E02D41E0D80112966C910995F8015E
:106E80008481982F9170E91237C082FDB5C0877F49
:106E9000D80114968C93B8C0B6E0EB1217C0EA8103
:106EA000FB81808181FF12C084E0569547958A95C9
:106EB000E1F7D8019A968C919A97841709F420C229
:106EC0009B966C929B979A964C93EBCEF80182819D
:106ED0009381DC01ED91FC910480F581E02DA3CE3E
:106EE000AA24A394B12C1ACF9581E91609F439CFBD
:106EF0008260848317821682AA94AB2889F7A090B7
:106F00006105B09062058501D12CC12C6C2DF60174
:106F1000EE0FFF1FE751FD4F20813181D8011D96F3
:106F20009C911D971E968C911E97891730F016968E
:106F30003C932E9315971E961C92F801868589170F
:106F400010F48F0D8687D80115964D915C91169798
:106F500017968D919C919A01281B390B37FF02C01F
:106F60002D5F3F4F3595279535952795211531058F
:106F700039F1F8015087478337FDA0C06486F801D6
:106F80008185882369F08481820F8483238592859B
:106F9000222309F49AC089170CF492C0891B8483B8
:106FA000F50182819381DC01ED91FC910680F781EE
:106FB000E02DD8011C962C911C9714964C910995A4
:106FC000055F1F4FCA94CD2809F074C00091610578
:106FD000109162055801E8EBAE0EB11CD5018C9101
:106FE0008F0D8C93712CF5018081803108F476C06F
:106FF000805180837394F7CFF80122853385283C34
:10700000310548F1877F8483F801E4808E2D8B7CE5
:1070100084838381811170CF80819181DC01ED9126
:10702000FC910190F081E02D40E0D80112966C9126
:1070300009958E2D887309F05FCFF80180819181C9
:10704000DC01ED91FC910280F381E02DD8011296D4
:107050006C91099551CF83FD0BC08F7E8483F8011D
:10706000848184FDCFCFD80111861086886811CF26
:1070700020853185283C310518F08F7E8483EFCF41
:1070800087FF02C08F778483F801848180618483C5
:1070900083818111E4CF80819181DC01ED91FC91AC
:1070A0000480F581E02DD80112966C910995D7CF17
:1070B000E58222CFCC24C394D12C28CF14865FCF75
:1070C00087FF6ECF890F84836BCF89171CF0915097
:1070D000948366CF87FF64CF148262CF772009F450
:1070E0009EC06801FCE9CF0ED11CE12C472C512C2D
:1070F000D60112968C911297E81608F05BC08E2C80
:10710000912C1396ED91FC911497E80DF91D808157
:10711000882361F11796ED91FC911897C401880FAF
:10712000991FE80FF91F80819181840D951D91832E
:1071300080836D917C9111970E2C02C07695679596
:107140000A94E2F715962D913C91D901A80DB91D2D
:107150004C91242F207F30E054E0359527955A95A7
:10716000E1F760FF05C08217930750F4E394C0CFA6
:107170004F7050E084179507C8F3841B950B02C02D
:10718000821B930B918380832F3041F06095709523
:10719000462F41706E2DC6010E942225D6011396FE
:1071A000ED91FC91E80DF91D80818F3FF9F281503E
:1071B0008083DCCFF801E255FF4F6281662359F1ED
:1071C0008481870D84837081B1812B2F207F30E0F3
:1071D00044E0359527954A95E1F7A22FBF7093813A
:1071E000492F407F50E014E0559547951A95E1F7F7
:1071F000721302C0841738F47B130DC09F70891777
:1072000050F07A1342C0841B8483B0836F3F19F01F
:107210008FEF860F82833596AE16BF0671F680918A
:107220006105909162050E949425E0916305F091BB
:10723000640582A9882399F080917505909176055F
:107240008F0D911D909376058093750520917305A0
:10725000309174058217930710F00E947B2980916A
:10726000780590916F058917A0F48F5F809378055A
:10727000E0E0F0E0EF2B09F426CC0E941C248823E8
:1072800009F41FCC0E9400001CCC891B848320833E
:10729000BDCF8913EDCF909177056FEF690F6830FF
:1072A00038F48DE595E00E94172A80917805DDCFAE
:1072B00083EF890F8830E8F490E0E1E8F6E4249168
:1072C000FC01EF51FD4F2083E1E7F6E42491FC013E
:1072D000E752FD4F2083880F991FFC01E753FD4FB4
:1072E0002081318187549D4FDC0111963C932E9370
:1072F000DCCF809170059813D8CF0E947B29D5CF21
:10730000E72C650114CCEF920F93FC0184819581E9
:10731000A681B78115962C9162131DC0DC01AD5476
:10732000BF4F442381F082E08C9384819581EE24C9
:10733000E394008521854FEF84569F4F0E9441259D
:107340000F91EF90089581E08C9384819581E12CD9
:1073500001852085F0CF84569F4F0F91EF900C94BC
:10736000222502970C948339EF920F93FC01A6819A
:10737000B78115962C911597621711F120851296F9
:107380004D915C91139714968C9190E0880F991F02
:10739000840F951FDC014D915C91062E02C056951D
:1073A00047950A94E2F740955095B42FB170EB2EB3
:1073B00084819581022F41E084569F4F0E94412590
:1073C0000F91EF90089502970C94B43902970C94A2
:1073D0004B2A0C944B2A0F931F93CF93DF931F924A
:1073E000CDB7DEB78C01DC011496ED91FC911597B9
:1073F000E255FF4F128281818F7080831496ED9148
:10740000FC91E255FF4F81E08083698341E050E0C9
:1074100064EF73E0CE0101960E942A3AC8010E94EF
:107420004B2A0F90DF91CF911F910F9108950297F2
:107430000C94EB39DC01CB01FC01F999FECF06C0BD
:10744000F2BDE1BDF89A319600B40D924150504022
:10745000B8F70895DC01A40FB51F4150504048F023
:10746000CB01840F951F2E910E943B3A4150504012
:10747000D0F70895262FF999FECF92BD81BDF89AD5
:10748000019700B4021639F01FBA20BD0FB6F89468
:10749000FA9AF99A0FBE0895A1E21A2EAA1BBB1BF5
:1074A000FD010DC0AA1FBB1FEE1FFF1FA217B307D0
:1074B000E407F50720F0A21BB30BE40BF50B661FE6
:1074C000771F881F991F1A9469F7609570958095AA
:1074D00090959B01AC01BD01CF010895A29FB00121
:1074E000B39FC001A39F700D811D1124911DB29FF8
:1074F000700D811D1124911D0895AA1BBB1B51E124
:1075000007C0AA1FBB1FA617B70710F0A61BB70B13
:10751000881F991F5A95A9F780959095BC01CD01B8
:107520000895052E97FB1EF400940E94A83A57FD7B
:1075300007D00E944C3A07FC03D04EF40C94A83AB2
:1075400050954095309521953F4F4F4F5F4F08958F
:1075500090958095709561957F4F8F4F9F4F0895BF
:10756000EE0FFF1F0590F491E02D09940F931F93E8
:10757000CF93DF938230910510F482E090E0E091A8
:107580008305F091840530E020E0B0E0A0E0309782
:1075900099F42115310509F44AC0281B390B243010
:1075A0003105D8F58A819B816115710589F1FB014F
:1075B00093838283FE0111C0408151810281138136
:1075C00048175907E0F04817590799F4109761F0E8
:1075D00012960C93129713961C933296CF01DF915B
:1075E000CF911F910F910895009383051093840507
:1075F000F4CF2115310551F04217530738F0A90196
:10760000DB019A01BD01DF01F801C1CFEF01F9CF24
:107610009093840580938305CDCFFE01E20FF31F85
:10762000819391932250310939832883D7CF2091B8
:10763000810530918205232B41F42091070130917F
:107640000801309382052093810520910501309136
:1076500006012115310541F42DB73EB740910901CE
:1076600050910A01241B350BE0918105F0918205B0
:10767000E217F307A0F42E1B3F0B2817390778F009
:10768000AC014E5F5F4F2417350748F04E0F5F1F68
:107690005093820540938105819391939FCFF0E0B1
:1076A000E0E09CCFCF93DF930097E9F0FC013297A5
:1076B00013821282A0918305B0918405ED0130E020
:1076C00020E01097A1F420813181820F931F209137
:1076D0008105309182052817390709F061C0F093C0
:1076E0008205E0938105DF91CF910895EA01CE17DD
:1076F000DF07E8F54A815B819E0141155105B1F72D
:10770000E901FB83EA8349915991C40FD51FEC1716
:10771000FD0761F4808191810296840F951FE90134
:1077200099838883828193819B838A83F0E0E0E060
:1077300012968D919C9113970097B9F52D913C91DC
:107740001197CD010296820F931F209181053091F0
:1077500082052817390739F6309751F510928405BC
:1077600010928305B0938205A0938105BCCFD3838B
:10777000C28340815181840F951FC817D90761F4D6
:107780004E5F5F4F88819981480F591F5183408315
:107790008A819B81938382832115310509F0B0CFC3
:1077A000F0938405E09383059ECFFD01DC01C0CFFB
:1077B00013821282D7CFDC0101C06D93415050403B
:0877C000E0F70895F894FFCFF3
:1077C800FF01047004000085058000040204010420
:1077D8000003040FF0000000005224B223DF239FAF
:1077E800241024EE2302240000000077268B2600B4
:1077F8000000004B284A284A283F2800000000C300
:107808002AB027CB278E278D279B29E939E939B458
:10781800398339EB39FEFF0000E639E639E339B13F
:1078280039173A564D4450565F317C315F564D44B6
:0478380050560A009C
:00000001FF
